:1000000013C4000049C4000047C4000045C40000F8
:1000100043C4000041C400003FC400003DC40000D0
:100020003BC4000039C400000C94CA2C0C94B22DBF
:100030000C94291331C400002FC400002DC400000B
:100040002BC4000029C4000027C4000025C4000000
:1000500023C400000C94A62C1FC400001DC4000083
:100060001BC4000019C4000017C4000015C4000020
:1000700013C4000011C400000FC400000DC4000030
:100080000BC4000009C4000007C4000005C4000040
:100090000C94B62F01C40000FFC30000FDC3000094
:1000A000FBC30000F9C30000F7C30000050109808D
:1000B000A101850319012AB700150126B700950192
:1000C00075108100C0050C0901A101850419012AE0
:1000D000A002150126A002950175108100C005013E
:1000E0000906A1018506050719E029E71500250184
:1000F0009508750181020507190029EF15002501F2
:1001000095F075018102050819012905950575010C
:100110009102950175039101C00660FF0961A1017B
:100120000962150026FF00952075088102096315F4
:100130000026FF00952075089102C005010906A15F
:1001400001050719E029E7150025019508750181CA
:10015000029501750881010507190029FF15002680
:10016000FF0095067508810005081901290515008D
:100170002501950575019102950175039101C00056
:100180000C55FFFFFF00000000000C00FFFFFF0008
:10019000000000000C80FFFFFF00000000000C00CA
:1001A0000000FF0000000000000000000000000050
:1001B000000000000000000000000000000000003F
:1001C00000000000000000000000007E0F00D4FFCF
:1001D000FFFFC70000007800000000000000002AB8
:1001E0002B280000000000000000000000000000BC
:1001F000000029000000002C1E3420212224342677
:1002000027252E362D3738271E1F2021222324256F
:10021000263333362E37381F0405060708090A0B24
:100220000C0D0E0F101112131415161718191A1B96
:100230001C1D2F3130232D350405060708090A0B34
:100240000C0D0E0F101112131415161718191A1B76
:100250001C1D2F3130354C09025B00030100A0FA50
:10026000090400000103010100092111010001221C
:10027000440007058103080001090401000203008E
:10028000000009211101000122220007058203203C
:100290000001070503032000010904020001030017
:1002A0000000092111010001226D000705840320CF
:1002B00000011201000200000008EDFE01E400014F
:1002C000010203011C037600690061006C003A0022
:1002D00066003600340063003200620033006300C1
:1002E00000001E034C0065007400730020005300E2
:1002F00070006C00690074002000450068003F0039
:1003000000001C0354006800610074002D004300CD
:1003100061006E0061006400690061006E00000011
:10032000040309042B0014001A000800150017002C
:10033000290004001600070009000A00E1001D0062
:100340001B000600190005002352E000E200E30054
:1003500021522C001C0018000C00120013002A006F
:100360000B000D000E000F003300340011001000D0
:1003700036003700380028002C002252500051006F
:1003800052004F0035021E021F02200221022202EB
:100390004C003A003B003C003D003E0001004000A4
:1003A000410042004300440001000100010001003F
:1003B00001000100230224022502260227024C002C
:1003C0003F002D022E022F02300231024500320280
:1003D000640201000100010001000100AB00AA005D
:1003E000A900AE0035001E001F00200021002200E1
:1003F0004C003A003B003C003D003E000100400044
:1004000041004200430044000100010001000100DE
:1004100001000100230024002500260027004C00D5
:100420003F002D002E002F0030003100450032002B
:10043000640001000100010001000100AB00AA00FE
:10044000A900AE000100007C0100010001000100D4
:1004500001000100010080748174010001000100AD
:100460000100010001000100010001000100010084
:1004700001000100010001000100010001004C0029
:100480000100010001000100010001000100010064
:100490000100010001000100010001000100010054
:1004A000010001002223252628292A2C2D2F303255
:1004B000333536383A3B3D3E4042434547494A4C46
:1004C0004E5051535557595A5C5E60626466686974
:1004D0006B6D6F71737577797B7D7F81838587897C
:1004E0008A8C8E90929496989A9C9E9FA1A3A5A781
:1004F000A8AAACAEAFB1B3B4B6B8B9BBBCBEBFC1AD
:10050000C2C3C5C6C7C9CACBCCCDCED0D1D2D2D337
:10051000D4D5D6D7D7D8D9D9DADADBDBDBDCDCDC4B
:10052000DCDCDDDDDDDDDCDCDCDCDCDBDBDBDADA0E
:10053000D9D9D8D7D7D6D5D4D3D2D2D1D0CECDCC85
:10054000CBCAC9C7C6C5C3C2C1BFBEBCBBB9B8B69A
:10055000B4B3B1AFAEACAAA8A7A5A3A19F9E9C9A25
:1005600098969492908E8C8A89878583817F7D7BF3
:1005700079777573716F6D6B6968666462605E5CD4
:100580005A5957555351504E4C4A4947454342409A
:100590003E3D3B3A3836353332302F2D2C2A292830
:1005A00026252322FFAA7F554000010101010101F8
:1005B000010101020202020202020202030303031A
:1005C00003030303040404040404040505050505EA
:1005D00006060606060707070707080808080909A8
:1005E00009090A0A0A0B0B0B0C0C0C0D0D0D0E0E53
:1005F0000E0F0F0F101011111112121313141415E6
:100600001516161717181819191A1A1B1B1C1D1D59
:100610001E1E1F20202122222324242526262728AF
:1006200029292A2B2C2D2D2E2F30313232333435DF
:10063000363738393A3B3C3D3E3F404142434445E2
:10064000464748494A4C4D4E4F50515354555658C1
:10065000595A5B5D5E5F616264656668696B6C6D6B
:100660006F7072737577787A7B7D7E8082838587E1
:10067000888A8C8E8F91939596989A9C9EA0A2A31F
:10068000A5A7A9ABADAFB1B3B5B7BABCBEC0C2C424
:10069000C6C9CBCDCFD1D4D6D8DBDDDFE2E4E7E9E4
:1006A000EBEEF0F3F5F8FAFDFF9D01930189017F70
:1006B0000100001E0F057F3F1F643214783C1E1E90
:1006C000140A05FD377A585A000004E6D6B44602EB
:1006D00000210116000000742FE5A3E002F10123C0
:1006E0005D003D8889C65436C3174FE4E20E167F7D
:1006F00084EBC5EC514B0AC693CBBF3859C3AD2F21
:100700006C7AE088B8CBF64B5D312A88D86F08C682
:10071000472490D28073F5E4ED82C989D459609B57
:100720006C50A14A30133032A4C2E07FF020634FF6
:10073000EE01DCFF47C68F80E793FF6CF89A412AF1
:10074000897152663CA5455D2950015D22FE13FD6D
:10075000D1AA9B696073A95D189F6DBA570384097C
:100760007794DA30ADB3DAC5579A3BB91FFC25DE72
:100770002BE1ACF9C0FB45A346F77D5EC616093BED
:10078000AAA0F2AEABA91BFDFDC449867C62651C24
:10079000B4BB2D23785E14339094A98F35EF6E6C23
:1007A0004EEA29476235791D123D39F83C4EE0AFDB
:1007B0004D4960593B9C7379C94DE44B925E7C2650
:1007C000A7961034C8DFE5004FD9E289988F3489A5
:1007D00055DB2DEA0A875BDFA3E0D0D1AB93C35092
:1007E00058165A1457FCBB7365725336DBADE0FBE9
:1007F000E9FAF12F3A82410EE8E8CE606D6A8D6A1F
:10080000899EE2E4D600007AEA1C8297094F2A000A
:1008100001BF02F2050000DA3AAD78B1C467FB020D
:100820000000000004595A0011241FBECFEFDAE087
:10083000DEBFCDBF04B603FE18C080914C0490917A
:100840004D04A0914E04B0914F048730904BA740C7
:10085000B04B59F410924C0410924D0410924E0477
:1008600010924F04E0E0F8E3099524E0A2E0B2E042
:1008700001C01D92AC34B207E1F712E0A0E0B1E094
:10088000E8E7F5E602C005900D92A230B107D9F76E
:100890000E94B0250C945B32B3CB9C01FB019A956E
:1008A00081159F4120F5832F8170B32FB270AA2745
:1008B000732F74706627532F5870442734FF0DC070
:1008C0008295807FAB2B09F08062672B09F08064F2
:1008D000452B09F0806809950895AB2B09F08260DB
:1008E000672B09F08460452BB1F38860F4CF80E07A
:1008F000F2CF8093E8030895292F983090F5863041
:1009000080F590E036E0239F800D911D1124282F63
:10091000277041E001C0440F2A95EAF723E096953D
:1009200087952A95E1F7FC01EE0FFF1FE80FF91FED
:10093000E95CFC4F20E030E070E05191DF01CB0139
:10094000022E02C0969587950A94E2F781708195F0
:100950008527842385278E932F5F3F4F23303105D2
:1009600061F70895292F983078F5863068F590E082
:1009700036E0239F800D911D1124682F677023E0BE
:10098000969587952A95E1F7FC01EE0FFF1FE80F7A
:10099000F91FE95CFC4F40E050E080E0219130E03D
:1009A000062E02C0369527950A94E2F72170332768
:1009B000042E01C0220F0A94EAF7822B4F5F5F4F8B
:1009C0004330510559F7089580E008958091F1036F
:1009D0009091F003981301C008958F5F8770FACF4C
:1009E000982F90958091E60389238093E6030895DC
:1009F0008091E503811531F01092E5031092EF0329
:100A00001092EE030895803E9105D9F1C8F4813328
:100A1000910509F482C048F48932910509F472C045
:100A20008A32910509F480C0089589339105E9F06F
:100A300082389105D1F08533910509F45EC008959F
:100A4000843E9105D9F148F4823E910539F1833E07
:100A5000910549F181EE90E00895863E9105C9F136
:100A6000873E910509F43EC008952091310423701A
:100A7000211164C02091320423FF14C089E290E068
:100A800008952091310420FD45C03091320430FF9B
:100A900009C024FD24C083EE90E008952091310424
:100AA00022FDF7CF08952091310422FD44C03091FA
:100AB000320430FD43C024FFF5CF11C02091320431
:100AC00021FFF0CF8091310484FD09C087EE90E0D2
:100AD00008952091310423FFE5CF24FFF7CF80E074
:100AE00090E008952091310423FD2BC03091320411
:100AF00031FFE1CF84EE90E008952091310425FF8D
:100B0000D1CFBCCF2091310425FD1EC020913204ED
:100B100023FFC8CF89E390E008952091310426FF98
:100B2000C1CF8AE290E008952091310426FFBACF28
:100B300081E390E0089582EE90E0089580EE90E0E9
:100B4000089586EE90E0089585E390E008959091F1
:100B5000310492FF10C041E0282F2471243009F0A5
:100B600040E031E0282F2871283009F030E04317A9
:100B700011F02CE0822793FF10C041E0282F247150
:100B8000243109F040E031E0282F2871283109F0A4
:100B900030E0431711F02CE082273091320430FF0F
:100BA00010C051E0282F2171213009F050E041E0C0
:100BB000282F2871283009F040E0541711F029E05F
:100BC000822731FF10C041E0282F2171213109F027
:100BD00040E031E0282F2871283109F030E0431738
:100BE00011F029E0822794FD877E08951F93CF930B
:100BF000DF9309DFEC01811522E5920708F052C06E
:100C0000811540E5940708F0CDC0803E910520F5A0
:100C10008D3C910508F0A1C0883A910570F4853AA1
:100C2000910508F097C081309105B9F10497813A98
:100C3000910598F1C0E0D0E030C0885A91094B97F7
:100C4000C8F7C85AD0E0CC0FDD1FCB56DE4F099055
:100C5000D881C02DD46421C0811550E49507B0F42B
:100C6000C11580E2D80708F0B3C0C83ED105A8F08E
:100C7000CE019A9581159F41E8F68D2F68DF182FD8
:100C8000CE019927C0DEEC01D12B07C09927BBDE2E
:100C9000CC27DF70C82BD92BD06ACE01DF91CF9142
:100CA0001F910895803842E59407C8F5803652E5D3
:100CB000950708F05BC0C03482E5D807D0F4C03295
:100CC00092E5D90708F04BC08C2F8695869520E2D7
:100CD000829FC0011124C37021E030E0A90102C04D
:100CE000440F551FCA95E2F7EA01C82BD92BDD68DE
:100CF000D4CF8C2F86958695877050E2859FC00152
:100D00001124C37021E030E0A90102C0440F551F37
:100D1000CA95E2F7EA01C82BD92BDC68BECF803C2C
:100D200052E5950758F48F71C03AD245A0F590E08E
:100D3000982F8827EC01C46FD06AAFCF805C9245B2
:100D4000809708F077CFDC2FCC27CC27DF71C06FDE
:100D5000D06AA3CFA497D064A0CFD0659ECFCF7127
:100D6000D0E0DC2FCC27C16FD06A97CF86958695CF
:100D7000877020E2829FC0011124C37021E030E01F
:100D8000A90102C0440F551FCA95E2F7EA01C82B1A
:100D9000D92BDA6882CFDBDEC82FD0E0DC2FCC275E
:100DA000D0627BCF8F71D3DE93E0CC0FDD1F9A959D
:100DB000E1F7CC27DF70282F30E084FF05C050E139
:100DC000859F900111243327C22BD32BD06965CF87
:100DD0008D2F8F71BCDE182FCE01992714DEEC0108
:100DE000D12BDECF80E00895F894E82FE295EF70E4
:100DF000F0E041A18F7021E030E0B90102C0660F40
:100E0000771F8A95E2F7CB01962F9095942391A3B3
:100E100092A1892B82A3789408950895CF92DF92AE
:100E2000EF92FF921F93CF93DF93172FE82FF0E0FD
:100E3000E755FA4F71110CC0E4918E2F7E2F6E2F63
:100E4000DF91CF911F91FF90EF90DF90CF900895A9
:100E5000E62EF12CC72ED12CF491EF2F86E0689F5F
:100E600090011124CFEFD0E0C901BE010E94633090
:100E7000AB01EE0CFF1C65E5649FC001659F900D02
:100E80001124E81AF90A6E2D660F6E0D7E01EC181A
:100E9000FD08FE9DD001FF9DB00D11248B2F169FE4
:100EA00070011124EF2CFF246E01CE18DF087601AB
:100EB000FE9D6001FF9DD00C11247E01E61AF10811
:100EC000B701169F7001179FF00C1124EF2CFF241F
:100ED000CE19DF09FC9F7001FD9FF00C11247F2DBE
:100EE00043305105C1F02C3F334058F44130510597
:100EF000B1F04230510509F0A2CFEB2F8F2D7F2F9B
:100F00009ECF4430510571F04630510509F497CF1A
:100F10007B2F8D2D94CF7D2DEB2F8F2F90CF7F2F7B
:100F2000ED2D8DCFEF2D7B2FF8CFCF93982F762FF0
:100F3000842FC22F692F72DF472F282F8091110134
:100F4000C81B8C2F90E0C6D0CF9108958091DD030F
:100F5000843028F4837084608093DD03089588389A
:100F6000E8F383708468F8CF21E030E0A90102C083
:100F7000440F551F8A95E2F7CA012091DC036115E1
:100F800061F0242B2093DC038091DB03806180934C
:100F9000DB0381E08093D702089580952823F2CF68
:100FA000CF93C82F8670863029F4C860C1FB6627AE
:100FB00060F904C0C77F60E0C111F8CF81E0D4DFE1
:100FC000C2FB662760F9C11101C060E082E0CCDF9E
:100FD000C3FB662760F9C11101C060E083E0C4DF94
:100FE0008C2FCF910895DCDF8093E903089521E0F1
:100FF00030E001C0220F8A95EAF78091E903822B45
:10100000F2CF21E030E0A90102C0440F551F8A95BC
:10101000E2F7CA0180959091E9038923E4CF90918A
:10102000EB03809589238093EB03282F27702111F0
:1010300010C0891771F09091320492FF0AC0869512
:1010400086958695DEDF1092EB031092ED031092E9
:10105000EC0308959091E90321E030E0F90101C02B
:10106000EE0F8A95EAF7D90102C0AA0FBB1F6A9555
:10107000E2F7EA2B01C0220F4A95EAF7892F8E2367
:10108000E81303C0892F822BAECF2095822F8923AE
:10109000FBCFE9EDF3E011828281846082830895C1
:1010A000E3E5F3E080E090E062E273E245E453E2DE
:1010B00027EB33E277836683518740873387228724
:1010C00097878687019670968830910599F70895DD
:1010D000229A0895FC01EE0FFF1FE80FF91FEC5A4A
:1010E000FD4F6183408322830895FA01309709F010
:1010F0000995089580910503811569F0E0912D030C
:10110000F0912E03309739F00190F081E02D309767
:1011100011F00995089580E00895A3E0B0E0E3E9B7
:10112000F8E00C9487309C01809152029091530218
:1011300082179307B1F03093530220935202E0914B
:101140002D03F0912E03309761F00084F185E02D9E
:10115000309739F083E089833B832A83CE0101965F
:1011600009952396E2E00C94A330A3E0B0E0EBEB0A
:10117000F8E00C9487309C018091500290915102CC
:1011800082179307B1F03093510220935002E091FF
:101190002D03F0912E03309761F00084F185E02D4E
:1011A000309739F084E089833B832A83CE0101960E
:1011B00009952396E2E00C94A33090914D01913073
:1011C00091F0A6E0B2E0EFEF90E02D91821751F0A0
:1011D000EF3F19F4211101C0E92F9F5F9630A9F765
:1011E000EF3FC9F408959091310497FFEACFE82FBB
:1011F000E695E695E695803FA8F7F0E0E45FFD4FC1
:10120000877021E030E001C0220F8A95EAF78281E1
:10121000822B828308950E2E000CFF0BEC5FFD4F96
:10122000F8CF90914D01913021F49091310497FDC8
:101230000CC0E6E0F2E09191891302C0DF011E923A
:1012400052E0EC30F507B9F70895E82FE695E695FA
:10125000E695803FC8F7F0E0E45FFD4F877021E03E
:1012600030E0A90102C0440F551F8A95E2F7CA0178
:101270008095928189238283089580914C010895FD
:101280002FB7F89460914C0270914D0280914E02FC
:1012900090914F022FBF08950F931F9380910503E4
:1012A000811521F0EDDF1F910F910895E9DF009185
:1012B0000103109102032091030330910403600F96
:1012C000711F821F931FEFCF0895FC019B01809136
:1012D0004202909143028617970740F0672B29F44A
:1012E0008091E8008E778093E800C90140E0009784
:1012F00041F4411106C08091E80082FF2FC080E0D8
:1013000008952091F0022115A9F12530A9F120912D
:10131000E80023FD2DC02091E80022FDECCF2091B4
:10132000E80020FFE4CF3091F3002091F200009715
:1013300019F02830310558F041E02830310509F026
:1013400040E02091E8002E772093E800D0CF419133
:101350004093F10001972F5F3F4FE9CF8091F0025A
:10136000811541F0853041F08091E80083FFC3CFC3
:1013700081E0089582E0089583E0089580913C0221
:1013800087FF13C08091E80082FF06C08091E800CB
:101390008B778093E80008958091F0028111F2CF5D
:1013A00008958091F0028115D9F38091E80080FFC3
:1013B000F8CF8091E8008E77ECCF2091E400309157
:1013C000E50095E6A9012091EC00822F817020FFB5
:1013D00006C08091E80080FF06C080E0089520915B
:1013E000E80022FD1AC08091F002811589F0853055
:1013F00089F08091EB0085FD0FC02091E4003091D1
:10140000E50042175307F9F29A95E1F684E0089552
:1014100082E0089583E0089581E00895E8EDF0E02A
:1014200080818E7F80831092E2001092DA00109209
:10143000E100A0EEB0E08C9181608C9380818F7789
:10144000808319BCA7EDB0E08C918E7F8C93808156
:101450008F7E808310923B020895E0912D03F091DE
:101460002E03309739F00284F385E02D309711F088
:1014700060E209950895FC01AC014C5F5F4F8FEF6E
:1014800061E39191892728E030E0982F990F87FF39
:1014900009C0892F862721503040B9F7E417F50796
:1014A00081F70895892FF7CF982F9093E900891736
:1014B00071F07091EC002091ED005091F00021FD51
:1014C00009C09F5F973089F78093E9000895762FD0
:1014D000242F50E03091EB003E7F3093EB003091B1
:1014E000ED003D7F3093ED003091EB0031603093A3
:1014F000EB007093EC002093ED005093F0002091EE
:10150000EE0027FDDECF0895A0E0B0E0EAE8FAE0C3
:101510000C948130C8EDD0E088818F7E8883E7ED20
:10152000F0E080818160808384E082BF81E08093ED
:101530003B0288818E7F888302EE10E0F8011082E2
:101540001092DA0081EEC82ED12CF601108288812B
:101550008F77888388818068888388818F7D88835E
:1015600019BC1092F00210923A021092CD02109221
:10157000390290EEE92EF12CF70180818B7F808378
:1015800088818160888342E060E080E08DDFF60141
:1015900080818E7F8083F80180818160808380815B
:1015A00088608083F70180818E7F8083888180615D
:1015B0008883CDB7DEB7E8E00C949D30E091F1036D
:1015C0009091F00327E0E91302C080E00895AE2F68
:1015D000B0E02E9FF0011124EE50FC4F3181361304
:1015E00006C03081381303C03581341304C0FD01B7
:1015F0003196E770E8CF81E0089535B13B7F25B1A2
:1016000024604FB7F89484E592E0FC010196508184
:1016100068E025B9000000C057FF35B9550F00003C
:1016200000C000C000C035B900C06A9591F752E013
:101630008837950751F74FBF8FE594E00197F1F791
:1016400000C00000089581E08093E00080E2809374
:10165000D8001092C9008FE19EE40197F1F700C015
:10166000000087E090EBDC0180934C0490934D04E4
:10167000A0934E04B0934F0488E19CE00FB6F89419
:10168000A895809360000FBE90936000FFCF0F93EA
:101690001F93CF93DF938B01EA019091F002943076
:1016A00051F58093E9008FEF9091E80095FD06C019
:1016B00095ED9A95F1F700008A95B1F78091E800D1
:1016C00085FF19C07ADE811111C08091E80085FD87
:1016D00006C08091E8008E778093E800F3CFF80190
:1016E00081918F018093F100219779F78091E80033
:1016F0008E778093E800DF91CF911F910F9108952D
:10170000792F603229F440E250E0682F82E0BFCFA9
:101710000895CF93DF93D82FC92F48E050E0682F6A
:10172000792F81E0B4DF88E0ED2FFC2FA4E4B2E054
:1017300001900D928A95E1F7DF91CF910895BC0158
:1017400040E250E084E0A3CFBC0143E050E084E0FD
:101750009ECFA0E0B0E0EFEAFBE00C947F30F82EE3
:10176000E92EB62EA72E8A01809136029AE0C92E64
:10177000D12C8A3018F0CC24C394D12CC1E0D0E015
:101780006B2D7A2D8F2D9E2DF8010995811116C094
:101790002196CC16DD0694F0CC9FC001CD9F900D14
:1017A000900D112420E030E045E34A95F1F7000068
:1017B0002F5F3F4F28173907B9F7E2CFCDB7DEB714
:1017C000EAE00C949B309091320492FB222720F99E
:1017D000281771F080FB92F99093320460913104E4
:1017E0007091320484E090E00E94E33182E017CCF3
:1017F00008951F93CF93DF93962F122F632F84307A
:10180000D8F49830C8F44630B8F4C42FD0E0CC0FE8
:10181000DD1F2CE0929FC00DD11D112490E6899F01
:10182000C00DD11D1124CE0189960E94C931612FAE
:10183000CE018A960E94C931DF91CF911F91089500
:10184000A0E0B0E0E6E2FCE00C947A30D82EFA0199
:10185000522EC32E780198E08902E0011124EF2B6B
:1018600079F5FE01ED5DFE4F86819781892B09F0A8
:101870004DC0E114F10411F1FE01ED5DFE4F8381D5
:10188000A82EB12CE816F10408F45701CD5DDE4F07
:101890006C817D81AB014A5C5B4F04E610E09501F1
:1018A00082E30E941D2F97FD2BC06C817D816A5CB5
:1018B0007B4FA501852D9C2D0E94883181E021C0A0
:1018C000DE01AD5DBE4F8C91A82EB12C481751059D
:1018D00008F45A01FE01ED5DFE4F81809280C40143
:1018E0008A5C9B4F3C01A5010E94883104E610E010
:1018F0009501A301682D82E30E94D12E97FFB1CFFD
:1019000080E0CDB7DEB7EFE00C949630D09236048D
:1019100060912401709125012091230130E0AB01F9
:101920004A5C5B4F04E610E082E30E94D12E97FFF1
:10193000A0CFE6CF8F929F92AF92BF92DF92EF92AD
:10194000FF920F931F93CF93DF9300D000D00F929D
:10195000CDB7DEB77B0101E010E09E012B5F3F4F6A
:1019600040E050E060E070E081E06ADF182F811510
:1019700009F442C08090FD029090FE02A090FF0208
:10198000B09000037DDCDD80681979098A099B0924
:10199000643671058105910528F488E394E06BDDD8
:1019A0008D1551F104E010E09E012F5F3F4F40E0A4
:1019B00050E060E070E082E043DF182F88E394E0BD
:1019C0005ADD8D1127C0111529F15ADC6093FD02F3
:1019D0007093FE028093FF029093000389819A81A5
:1019E000AB81BC818093F9029093FA02A093FB0231
:1019F000B093FC0281E00FC08091380490913904CB
:101A0000A0913A04B0913B0489839A83AB83BC8351
:101A10001111E4CF80E04091F9025091FA026091F7
:101A2000FB027091FC02F701408351836283738350
:101A30000F900F900F900F900F90DF91CF911F910B
:101A40000F91FF90EF90DF90BF90AF909F908F909D
:101A50000895A4E0B0E0EFE2FDE00C948130C09086
:101A6000F502D090F602E090F702F090F80208DC60
:101A70006C197D098E099F0911E064367105810595
:101A8000910508F109DCDC01CB010296A11DB11D15
:101A900089839A83AB83BC8300E010E020E030E0D0
:101AA00044E050E0BE016F5F7F4F83E0C9DE182F36
:101AB000811549F0E5DB6093F5027093F60280939F
:101AC000F7029093F802812F2496E8E00C949D3061
:101AD0008F929F92AF92BF92FF920F931F93CF93DB
:101AE000DF93CDB7DEB72C970FB6F894DEBF0FBEED
:101AF000CDBF88E0EDEDF3E08E010F5F1F4FD80101
:101B000001900D928A95E1F73091D9032091DA0383
:101B10008091DB039091DC0339872A878B879C8730
:101B2000F82E8090F1029090F202A090F302B09013
:101B3000F402A6DB681979098A099B09F02FE12FC5
:101B4000643671058105910510F4F114A9F000E0E7
:101B500010E020E030E04CE050E06F2F7E2F84E07A
:101B60006FDE811561F08CDB6093F1027093F202FD
:101B70008093F3029093F4021092DB0381E02C96A1
:101B80000FB6F894DEBF0FBECDBFDF91CF911F918E
:101B90000F91FF90BF90AF909F908F9008950F93FB
:101BA0001F93CF93DF93843030F5683020F54630B3
:101BB00010F5C42FD0E0CC0FDD1F2CE0629FC00DCC
:101BC000D11D112430E6839FC00DD11D1124CE01FB
:101BD00089960E94A831082F10E0102F0027CE010F
:101BE0008A960E94A8319801282BC901DF91CF91D4
:101BF0001F910F91089580E090E0F8CF462F672F56
:101C00002091090330910A03232B81F4703F39F4AA
:101C1000403F61F480910703909108030895783064
:101C200028F4463018F4843008F4B9CF80E090E00E
:101C30000895A0E0B0E0EFE1FEE00C9482307C017A
:101C40000091E9038091E803082BC3E0D0E010E0A5
:101C5000C8010C2E02C0959587950A94E2F780FD85
:101C600009C02197A8F7D12C8D2DCDB7DEB7E7E0BD
:101C70000C949E30DC2EB7018C2FC0DF0E94F6053D
:101C8000019779F3F1CF0F931F93CF93FC018581D7
:101C900000811181811581F0611571F0C801C9DFE2
:101CA000C82F682FC8010E947C04B8018C2FA6DFC2
:101CB000CF911F910F910895C8010E94B204C82FBF
:101CC000F4CFCF93DF93D82FC92FB3DF6D2F7C2FA5
:101CD00095DF0E94F605DF91CF910895FC01848184
:101CE000811599F080819181ECDF282F92959F706A
:101CF000963099F060F4925F9F70923030F4203FFC
:101D0000B1F038F481E0283E38F080E008959A5F21
:101D1000F3CF81E0243FC9F7089591E0213F09F016
:101D200090E081E0283E08F080E0892B089581E072
:101D30000895382F292FCB01A32FB22F873022E00F
:101D40009207A105B10520F487509E4F0C94A8314D
:101D500080E0089585E290E00E94A831833589F4FF
:101D600086E290E00E94A8318B3459F487E290E03B
:101D70000E94A83191E08E3009F090E0892F8170A7
:101D8000089580E0FCCFA5E0B0E0E9ECFEE00C9423
:101D90007B308091DD0380FF0CC0A090C802B09022
:101DA000C902A114B104B9F428DC2596EEE00C9424
:101DB00097301091130180911401181770F78091DA
:101DC0001101912F981B892F20E040E060E090E006
:101DD00081D91F5FF0CF8091DD0380FFE5CFC12C5B
:101DE000D12C66246394712C8091DC0393010C2C1C
:101DF00001C0220F0A94EAF78223811559F1F501F7
:101E0000E590F590E114F10479F245E050E0B70176
:101E1000CE0101960E94653189818F3FD9F0882ECD
:101E2000912C0A81080F1127111F0D30110514F094
:101E30000CE010E08016910624F095E0E90EF11C0C
:101E4000E4CF94014D816C818B816FD88FEF881A1C
:101E5000980AF0CF82E0A80EB11C9FEFC91AD90AE8
:101E600088E0C816D10409F0BFCF9ECFEF92FF9251
:101E70001F93CF93DF93EC0110E0EE24EA94F12C52
:101E800060911501161768F07EDF8C819A8190FFB2
:101E90001DC08F5F8C83DF91CF911F91FF90EF90DA
:101EA000089520911301210F3327331F70E0C701DC
:101EB0000E94BA30962F8C814091E0036091DF033D
:101EC000199F800D112431D81F5FDACF8150E2CFE6
:101ED0001F93CF93DF93EC018C81811109C081E0C6
:101EE0008C831092BC0292E09093050180930401D0
:101EF0001091130180911401181740F110E06091C6
:101F00001501161778F13FDF809104019091BC0212
:101F1000980F9093BC0220910501280F2093050192
:101F2000121654F4209115012150330B092E001C78
:101F300000089217030634F08195809304018130E4
:101F400009F41C82DF91CF911F91089580911101B6
:101F5000912F981B892F20E040E060E090E0BAD8F4
:101F60001F5FC8CFE12FF0E070E0CF010E94BA30D0
:101F700020911301820F9091BC02092E001C0008D1
:101F8000E917F005A4F090910501092E001C000846
:101F90009E170F0664F0282F30E04091E003609117
:101FA000DF038091DE030E9495071F5FA8CF909109
:101FB0001101891B20E040E060E090E08BD8F5CF74
:101FC000EDEDF3E080818E7F808363D8E9EDF3E06F
:101FD000828181608283D7CE0F931F93CF93DF934B
:101FE000D82F162F042F8091DD03C091130180FD9F
:101FF00010C0DF91CF911F910F9108958091110131
:102000009C2F981B892F202F412F6D2F90E062D895
:10201000CF5F80911401C81788F3B5DEEACF982FFF
:10202000762F842F2091DD0320FF08C0692F0E94A6
:102030000E07962F672F482F892FCECF0895CF9365
:10204000DF93EC01EC81F0E0EC55FB4F4491EDEDBA
:10205000F3E062818181E3DF8C818F5F8C83DF918C
:10206000CF910895CF93DF93EC01EDEDF3E0438141
:1020700062818C81D4DF8C818F5F8C83DF91CF91E3
:102080000895AAE0B0E0E7E4F0E10C947C30A09081
:10209000EE02B090EF0281E090E09093EF02809327
:1020A000EE02812C912CE12C6401F12C14C0F8017A
:1020B00025913591472D6F2D8E2D9BDB0E5F1F4F88
:1020C000739486E07812F3CF86E0C80ED11CF394A7
:1020D00088E0F81639F08601000F111F0C5D1C4FC7
:1020E000712CE5CFE39480E3880E911C84E0E81224
:1020F000DBCF1A8219821C821B821E821D821886E7
:102100001F8288EC90E09A87898709EA11E04AE00B
:1021100050E0B801CE0101960E94E731065F1F4FE3
:10212000093F81E0180799F7B092EF02A092EE0202
:102130002A96EDE00C949830A0E0B0E0E2EAF0E1FD
:102140000C947930FC016280448081E08483E4EA6D
:10215000F4E07490E3E2F5E0E491C091E003C69509
:10216000C158D0E0CC0FDD1FCD2FDD27812C25E01D
:10217000922EAA24AA94B12C55245A94E719EE2E33
:10218000F12C80911501881630F0FDDDCDB7DEB75A
:10219000E0E10C949530C82CD12C83E0681658F4FB
:1021A000989CF0011124E058FD4F8091DE0380835C
:1021B0008091DF03818341101CC09C9CF0019D9C99
:1021C000F00D1124E058FD4F13821282809113010B
:1021D0009601280F311D9C9CF0019D9CF00D11244F
:1021E000E058FD4F4281618180810E949507839470
:1021F000C8CF9C9C80019D9C100D112400581D4F40
:10220000F80183818115F1F081508383589EC001CC
:102210001124648170E00E946330FB01FF27EC55BC
:10222000FB4F8491E82FE7195E9EC0011124B7018E
:102230000E9463308091E003689FB0011124F8018F
:102240007283C4CF0E945731B5010E94BA308C17F7
:102250009D070CF0BBCFF3E06F1698F00E9457314A
:10226000B5010E94BA30F80180830E945731209155
:10227000DF032695622F70E00E94BA30280FF80124
:1022800021839C9CF0019D9CF00D1124E058FD4F92
:1022900012828091E003893C58F088EC9C9CF0010C
:1022A0009D9CF00D1124E058FD4F848383838ECFD5
:1022B0008431A0F784E1F2CF0F93CF93DF93CDED7C
:1022C000D3E0488159816A817B8188E090E00E9457
:1022D000DB31288139814A815B816C817D818E81EE
:1022E0009F8100E20E94F530622F83E290E00E941D
:1022F000C931DF91CF910F910895EDEDF3E085E0C5
:10230000808311828FEF828383831482E9EDF3E06F
:102310008281836082838DED93E0CECF8091E10353
:10232000833018F48F5F8093E1038DED93E0C4CF89
:102330008091E103811519F081508093E1038DEDC7
:1023400093E0BACFA0E0B0E0E8EAF1E10C9482308B
:10235000C82F062F142FD22E3091DD0330FF34C04A
:102360008091DE038C1308C09091DF03961304C0A4
:102370009091E003941729F09091DB039260909381
:10238000DB03232F26952695E22FF0E0E959FE4F37
:1023900090819093D9033C7F3430D9F46C2F702F07
:1023A000812F0E940E07962F672F482F892F14DE4A
:1023B0008C2F8093DE030093DF031093E003D1148E
:1023C00019F08DED93E078DFCDB7DEB7E7E00C9440
:1023D0009E30923019F41091E003EACF963049F321
:1023E000993039F3923121F7EEEEE20F2170E22EAF
:1023F000E695F0E0EC55FA4FD491F12C609115017F
:10240000F61610F0C0DCD4CFFD9EC001112470E0A0
:102410000E9463308C2FE1100CC0860F20911301B5
:102420002F0D3327331F412F602F0E949507F39400
:10243000E5CF861BF3CFEDEDF3E0818121E0438111
:102440006281885F7FCFEDEDF3E0818121E0438100
:102450006281885077CFEDEDF3E0628121E1620F78
:1024600008F46FEF21E0438181816CCFEDEDF3E063
:10247000628121E1621B08F460E021E043818181F7
:1024800061CFEDEDF3E0438121E1420F08F44FEF1E
:1024900021E06281818156CFEDEDF3E0438121E1BE
:1024A000421B08F440E021E0628181814BCF282F5C
:1024B000CB01283070F44AE0249F90011124B90127
:1024C00067557E4F4AE050E00E94983180E090E0EE
:1024D00008958FEF9FEF0895AAE0B0E0E2E7F2E100
:1024E0000C9487309C0197558115914068F4BE018A
:1024F0006F5F7F4F822FDBDF892B31F489859A85CF
:102500002A96E2E00C94A33088EC90E0F9CFA0E1A9
:10251000B0E0EDE8F2E10C947930FE01319680E113
:10252000DF011D928A95E9F701E210E099EFA92EEB
:10253000BB24B39427E0422E22E0522E612C712C52
:102540004F0173016201B1E14B1651046104710442
:102550001CF080E1C82ED12CA601B501C4010E9457
:10256000BA31AC0CBD1C0D2C000CEE08FF084C1849
:102570005D086E087F080150104019F76096E0E191
:102580000C9495306FEF85E290E00E94C9316FEFB7
:1025900086E290E00E94C9316FEF87E290E00E94EE
:1025A000C93160E088E290E00E94C9316ADDAFDFA6
:1025B00063E585E290E00E94C9316BE486E290E039
:1025C0000E94C9316EE087E290E00C94C9318F928D
:1025D0009F92AF92BF92CF92DF92EF92FF920F93B2
:1025E000CF93DF9388E090E00E94B0314B015C0113
:1025F000CDEDD3E068839982AA82BB821C821D82C2
:102600001E821F8283E290E00E94A831282F30E0D2
:1026100040E050E060E070E080E090E000E20E9486
:10262000DA30282939294A295B29288339834A83C2
:102630005B836C837D838E839F83DF91CF910F912A
:10264000FF90EF90DF90CF90BF90AF909F908F90D2
:1026500008951F921FB61F9211248F939F93AF93DB
:10266000BF938091CA02811113C080914C02909156
:102670004D02A0914E02B0914F024196A11DB11D95
:1026800080934C0290934D02A0934E02B0934F0260
:10269000BF91AF919F918F911F901FBE1F90189572
:1026A0002FB7F89480914C0290914D02A0914E0268
:1026B000B0914F022FBF0895CF93DF93C091E603EF
:1026C0008091EA03C82B8091E503811501F1E8DFD1
:1026D0002091EE033091EF03821B930B88389341D6
:1026E00010F00E94F804D091E50380914D018130F3
:1026F00021F48091310487FD0EC086E026E032E0AF
:1027000090E0815060F491110E94F804CD2B8C2F41
:10271000DF91CF9108958EE12EE032E0F1CFF90103
:1027200041919F01411569F39F5FEBCF80914D016E
:10273000813061F58091310487FF28C0BDDF80932F
:102740000D0240E250E06DE073E08CE092E00E9408
:102750007B31892BD1F080E2ECE0F2E0ADE0B3E038
:1027600001900D928A95E1F7E0912D03F0912E03EF
:10277000309759F00480F581E02D309731F086E0F4
:1027800080930C028CE092E00995089595DF809388
:10279000040248E050E06FE273E084E092E00E94BF
:1027A0007B31892B91F388E0E4E0F2E0AFE2B3E023
:1027B00001900D928A95E1F7E0912D03F0912E039F
:1027C000309719F30280F381E02D3097F1F284E025
:1027D00092E0DACFCF93C82F8115C9F08CEF8C0F20
:1027E000813A90F580914D01813021F4809131043E
:1027F00087FD0FC0E6E0F2E08191C81701F122E009
:10280000EC30F207C9F78C2F0E94DD088FDFCF91E3
:102810000895EC2FE695E695E695F0E0E45FFD4F30
:10282000828190E04C2F477021E030E002C0220FFF
:10283000331F4A95E2F782239323892B21F38C2FB0
:102840000E94110973DFDFCF80E28C0F883068F4BB
:10285000C77081E090E001C0880FCA95EAF7C09187
:10286000E603C82BC093E603D1CF8BE58C0F8330F2
:1028700038F42C2F2452330BC9010E948D08C7CF86
:10288000C85ACB3120F6EC2FF0E0EE0FFF1FE553D6
:10289000FE4F808191810E94B508B9CF811521F149
:1028A0009CEF980F913A18F40E9411093FCF90E2E3
:1028B000980F983050F4877091E001C0990F8A9575
:1028C000EAF7892F0E94F004F1CF9BE5980F93302F
:1028D00020F480E090E00C948D08885A8B3120F42D
:1028E00080E090E00C94B50808951F93CF93DF9398
:1028F000182FEB016FDF209731F4812FCFDFDF91AD
:10290000CF911F9108958FE99FE00197F1F700C0E3
:1029100000002197F0CFA0E0B0E0E1E9F4E10C94F1
:102920008030EC018881811509F1813009F045C0C2
:102930008981813051F48A81239660E570E0893382
:1029400011F060E070E0D1DFEDCF823021F48A81B8
:10295000239640DFE7CF833021F48A8123969EDFE0
:10296000E1CF843041F022968111DCCFCDB7DEB7C4
:10297000E9E00C949C308A81239620E030E09AE0D4
:10298000682F6053770BAB016A30710560F0211539
:10299000310551F3EFE9FFE03197F1F700C0000096
:1029A00021503109F4CF929FB001939F700D1124F3
:1029B0009A01260F371F8991E3CFE82FF0E0E95203
:1029C000FE4FB490282F26952695269530E0F901E4
:1029D000E953FE4FE4908770F12C082E02C0F59465
:1029E000E7940A94E2F7E0FAEE24FF24E0F8F90114
:1029F000E954FE4FC490D12C082E02C0D594C79440
:102A00000A94E2F7C0FACC24DD24C0F8F901E955B4
:102A1000FE4F049110E002C0159507958A95E2F7E4
:102A200001701127E114F10411F081EED3DEC1141D
:102A3000D10411F086EECEDE60E070E08B2D55DF24
:102A4000C114D10411F086EE29DFE114F10411F074
:102A500081EE24DF0115110521F060E070E08CE2C9
:102A600044DF21965FCF811531F09091E603892BE9
:102A70008093E6035BCE0895811519F00E94F0045F
:102A800055CE0895811531F09091EA03892B8093FA
:102A9000EA034CCE0895811539F080959091EA03B0
:102AA00089238093EA0342CE08951092E603809131
:102AB0004D018130B1F48091310487FF12C0EEE006
:102AC000F2E08EE1DF011D928A95E9F780E090E067
:102AD0000E948D0880E090E00E94B5081092EA0301
:102AE00025CEE6E0F2E086E0EDCFDFDF2FEF84E3F6
:102AF0009CE0215080409040E1F700C0000088E158
:102B00009CE00FB6F894A895809360000FBE909358
:102B10006000FFCFAAE2B0E0E0E9F5E10C94863076
:102B20008CE392E0FC0101962091F100208322E0E9
:102B300084349207B9F780913D02893009F459C075
:102B4000C8F4823009F4B6C0833009F485C08130FE
:102B500089F18091E80083FFEAC080913C02909166
:102B60003D029A3008F0E3C0E92FF0E0E35AFD4C53
:102B70000C94CD308A3009F48CC08B3051F78091A1
:102B80003C02813231F78091400290914102892BC1
:102B900001F78091E800877F8093E8000E94BE09DA
:102BA00081E090913E02911101C080E080934D013F
:102BB0007CDFCFCF80913C02813A59F68091E800CA
:102BC000877F8093E8008091400290914102892B99
:102BD00061F060E080E090E070E00E946509809123
:102BE000E8008B778093E800B4CF68E084E492E05B
:102BF000F3CF80913C02813209F0ABCF809140024B
:102C0000909141028D7F892B09F0A3CF8091E8003C
:102C1000877F8093E8008091E80082FF18C0909140
:102C2000F3008091F200029731F48091F10081303D
:102C300011F0863021F48091F10080934C01809155
:102C4000E8008B778093E8000E94BE0982CF8091D4
:102C5000F0028111E0CF7DCF80913C02813A09F0F2
:102C600078CF8091400290914102892B09F071CF79
:102C70008091E800877F8093E8008091E80080FFE2
:102C8000FCCF80914D018093F1008091E8008E7718
:102C9000D9CF80913C02813209F05BCF8091E8006E
:102CA000877F8093E8000E94BE0980913F02809355
:102CB0004B014FCF80913C02813A09F04ACF80917D
:102CC000E800877F8093E8008091E80080FFFCCFD8
:102CD00080914B01D8CF803889F0823841F58091BE
:102CE00040028F70873018F58093E9008091EB00E7
:102CF00085FB882780F91092E90006C08091CD02FB
:102D0000880F90913902892B9091E800977F9093DA
:102D1000E8008093F1001092F1008091E8008E7736
:102D200023C0811116C080913E02813011F1809143
:102D3000E80083FF0AC08091E800877F8093E80065
:102D40008091EB0080628093EB00AA96E3E00C9404
:102D5000A230823061F780913E02811589F0109295
:102D6000E9008091E800877F8093E8000E94BE0917
:102D7000DECF81E0933009F080E08093CD02EFCF89
:102D8000809140028F702FEF280F263080F68093BD
:102D9000E9002091EB0020FFE2CF933031F48091E5
:102DA000EB0080628093EB00DACF9091EB009061B2
:102DB0009093EB0021E030E0A90102C0440F551FC1
:102DC0008A95E2F74093EA001092EA008091EB00C6
:102DD0008860E8CF8111ABCF10913E021F778091C0
:102DE000E3008078812B8093E3008091E800877F67
:102DF0008093E8000E94BE098091E80080FFFCCF2C
:102E00008091E30080688093E30083E0111101C0AA
:102E100082E08093F0028BCF8058823008F087CF19
:102E200080913E0290913F028C3D53E0950799F5C9
:102E300083E08A838AE289834FB7F894DE01139690
:102E400020E03EE051E2E32FF0E050935700849100
:102E500020FF03C082958F703F5F8F708A30C8F06B
:102E6000895C90E08D939D932F5F243161F74FBF74
:102E70008091E800877F8093E8006AE270E0CE01ED
:102E800001960E9465098091E8008B778093E800A5
:102E90004ECF805DE6CF292F33272330310509F44B
:102EA0004EC078F52130310509F488C08BE590E0FB
:102EB000E7E5F2E02230310509F039CF2091E80052
:102EC000277F2093E800209142023091430282172D
:102ED000930708F49C0140E02115310509F073C007
:102EE000411171C08091E80082FDCDCF8091F00248
:102EF000811549F2853039F28091E80083FFF2CFE5
:102F0000C2CF80914002909141022132310509F4F3
:102F100046C02232310509F00ACF8330910508F00E
:102F200006CFFC01EE0FFF1FE55AFE4F0190F08126
:102F3000E02D885A9E4FDC018C9190E010C09C01DE
:102F40003327823021F12330310568F4232BB9F483
:102F5000E0E2F3E0E4918E2F90E0E0E2F3E000970E
:102F600009F4E5CEABCF2330310509F0E0CEE4EC37
:102F7000F2E0E4918E2F90E0E4ECF2E0F0CFE2E0BA
:102F8000F3E0E4918E2F90E0E2E0F3E0E8CFE2EEB0
:102F9000F2E0E4918E2F90E0E2EEF2E0E0CF8330B9
:102FA000910508F0C4CEFC01EE0FFF1FEF59FE4F54
:102FB0000190F081E02D89E090E080CF82E190E007
:102FC000E2EBF2E07BCF8091F002811509F45BCF58
:102FD000853009F458CF8091E80083FD54CF80916B
:102FE000E80082FD7FCF8091E80080FF75CF90914F
:102FF000F3008091F2002115310519F08830910518
:1030000050F041E0089709F040E08091E8008E77A9
:103010008093E80061CF44914093F10031962150B4
:1030200031090196E8CF803809F081CE8091E8001F
:10303000877F8093E80080913A028093F1006DCE03
:10304000811175CE10913E02123008F070CE809141
:10305000E800877F8093E80010933A020E94BE093F
:103060001115F9F084E08093F00242E061EC81E018
:103070000E94540A42E261EC84E00E94540A42E257
:1030800061EC82E00E94540A42E260EC83E00E941C
:10309000540A8091F002843051F482E080934E0112
:1030A00046CE8091E30087FDDDCF81E0DCCF81E07B
:1030B000F5CFCF93DF93EC014A855B856E857F85E5
:1030C0000E9475089B8190958091EA0389238093E3
:1030D000EA038C810E94F00429DB86E0FE01119254
:1030E0008A95E9F7DF91CF910895CF93DF93EC01B3
:1030F0008D8181FD16C082608D838091EA039B8162
:10310000892B8093EA038091E6039C81892B80932D
:10311000E6030CDB488559856E857F85CE010E94CC
:1031200075081092D4031092D3038D8180FD02C0E4
:10313000CE01BFDFDF91CF910895962F2091320409
:1031400022FF0FC0682F660F660F660F692B609312
:10315000EB030E94F707A4DA9093ED038093EC034E
:1031600008950C94F7079091E503292F2823211542
:1031700059F0809589238093E503811531F090DA29
:103180008093EE039093EF03089580E090E0F8CFF2
:1031900080910503811509F083CA0E944C09CB0177
:1031A00008956091DD036695669570E04BE050E010
:1031B00086E091E00E946E31892B19F481E08093C2
:1031C000DA03E6DF9093DC028093DB028091DB037D
:1031D00084608093DB0308959091DD0390FF31C0FC
:1031E000811581F1823280F58F73880F880F90915D
:1031F000DD039370892B8093DD038091DB03816075
:103200008093DB03611519F08DED93E055D8609143
:10321000DD036695669570E04BE050E086E091E056
:103220000E946E31892B91F00E94490881E08093C1
:10323000DE0220E04091E0036091DF038091DE0335
:1032400081C8089581E0D1CF81E2CFCFAADFEECF50
:103250008091DD03869586958F5F823208F081E04C
:1032600061E0BACF8091DD03869586958A9509F451
:1032700081E261E0B1CFCF93DF93EC0111DA8C1BD7
:103280009D0BDF91CF910895A0E0B0E0EAE4F9E171
:103290000C948230162FD72FC42FD22E811599F07F
:1032A0004093D703FDD99093380280933702C770BB
:1032B00081E001C0880FCA95EAF7D5DBCDB7DEB74C
:1032C000E7E00C949E309091D703491334C0E0900E
:1032D0003702F0903802E4D99C012E193F09790198
:1032E000812F9D2FF9D8E816F90628F5D0E2DD0DDB
:1032F000CD1591F0C77011E0812F01C0880FCA95DC
:10330000EAF7BADBD83040F48D2D877001C0110F79
:103310008A95EAF7812FA7DB60E070E0802FE5DA7D
:10332000D83060F62D2D277081E001C0880F2A95D6
:10333000EAF7A2DBC3CFC77081E001C0880FCA954E
:10334000EAF7F7CFA8E0B0E0E8EAF9E10C947930C9
:103350005C01DC0114968C91811509F412C261E0C4
:10336000C5010E94430E8C01F5018581811529F16B
:103370008091D3039091D4030097F9F008171907AF
:10338000E1F0FC01FF27887F9927892B09F077C09E
:1033900044E0EE0FFF1F4A95E1F7ED5AFC4F85819F
:1033A0008460858311830083CF019FDE1092EA033E
:1033B00061E0C5010E94430E8C01D50115968C91E8
:1033C000811509F4EBC0980137572038310508F012
:1033D00094C1003108F0C4C166E072E080E090E082
:1033E0000E94990E8111BCC1C12CD12C7601011112
:1033F00049C004E09E012F5F3F4F4901D401E02FF7
:103400001D92EA95E9F726013701FFEF4F1A5F0A8F
:103410006F0A7F0AC701B6010E94990E8983811540
:1034200009F49EC1813009F0B6C0A70196012E5F54
:103430003F4F4F4F5F4F2D833E834F835887C301CC
:10344000B2010E94990E182F8A83811509F488C150
:103450008FEF810F833080F56D817E818F8198851C
:103460000E94990E8B83811511F0C40154DA260154
:10347000370133E0430E511C611C711C4DC0E0E06C
:10348000F0E08DCFB7E0CB16B2E0DB06E104F1044B
:1034900009F466C1C701B6010E94990EEFEFCE1A7A
:1034A000DE0AEE0AFE0A8111EDCF0150A0CF4D8059
:1034B0005E806F80788430C08BEF810F8330A8F5F9
:1034C0002601370143E0440E511C611C711C6D81C3
:1034D0007E818F8198850E94990E8B838115E1F002
:1034E000C301B2010E94990E8C83811571F08B810A
:1034F0009C8181305FEF950710F0982F8827163058
:1035000071F0173079F00E9417232601370134E05B
:10351000430E511C611C711C730162016FCF0E942C
:10352000B322F3CF0E94E522F0CF143009F0BFCFD1
:103530006D817E818F8198850E94990E182F2601BA
:10354000370184E0480E511C611C711CC701B60193
:103550006D5F7F4F8F4F9F4F0E94990E111509F499
:10356000FFC0811509F4FCC08150990B4FEF489FB3
:103570009001499F300D1124A12FA150BB0B2A0FA0
:103580003B1F2150310940F2EFE9FFE03197F1F79D
:1035900000C00000F6CFC401BED9BECF011527E59B
:1035A000120708F476C0011538E5130708F0ABC020
:1035B000780147E5F41A69E473E08E2D0E945712F2
:1035C000892B31F5C70124E0880F991F2A95E1F76F
:1035D000FC01ED5AFC4F2281213009F07AC0209184
:1035E000490330914A03232B99F020914B033091EA
:1035F0004C03232B69F020914D0330914E034091F1
:103600004F0350915003242B352B232B09F46BC00F
:10361000680188EFC822DD24C114D10409F0A0C0DC
:10362000F801FF2794E0EE0FFF1F9A95E1F7DF0105
:10363000AD5ABC4F7D01D50115968C91E85AFC4FCF
:10364000908180FB90F99083811509F467C028D898
:103650009093D6038093D503F70182818F5F828395
:103660008091EA039091E603892B83838091E5039F
:1036700084834681578166857785C7010E947508D6
:10368000D70115968C9181FF6801D092D403C09226
:10369000D303F5018581811509F4A1C41092D703E4
:1036A000980130572332310508F0A7C484E090E038
:1036B0000E94B5319093320480933104F801E150B7
:1036C000F047E232F10508F084C0E959FD4C0C9452
:1036D000CD30223009F09CCF20914D0330914E0324
:1036E000232B09F495CFFC01E85AFC4F20812E7F53
:1036F00020838D5A9C4FF9DC8BCF980137552115CB
:10370000314008F485CFF801E851FC47E730F10576
:1037100008F0BFCFE757FD4C0C94CD30F70144853E
:10372000558566857785C7010E947508D70115966E
:103730008C9181FFAECFC701BCDC8091D303909107
:10374000D4030817190709F0A4CF1092D4031092DC
:10375000D3039FCF06E221EE41EE6AE17CE794DDE0
:103760008091EB038770811561F0D50115968C91DE
:10377000811539F08091320482FF03C082E00E94FB
:103780000F082896E0E10C94953007E225EE45EE0F
:103790006BE17CE7E4CF06E221EE40EE68E17CE7F6
:1037A000DECF07E225EE44EE69E17CE7D8CF06E202
:1037B00021EE42EE6CE17CE7D2CF07E225EE46EE49
:1037C0006DE17CE7CCCF08E221E045EE6EE17CE7DD
:1037D000C6CF8091310481608093310460913104BF
:1037E0007091320484E090E00E94E3315ED9B8CF5A
:1037F00080913204886080933204F0CF809131044C
:103800008260EACF809131048460E6CF80913104F8
:103810008860E2CF809132048160EDCF80913204E4
:103820008260E9CF809131048061D6CF80913104EC
:103830008062D2CF809131048064CECF36D980911E
:1038400031048068C9CF809131048C60C5CF8091EC
:1038500032048360D0CF809131048E7FBDCF8091C0
:103860003204877FC8CF809131048D7FB5CF80919E
:1038700031048B7FB1CF80913104877FADCF8091B0
:1038800032048E7FB8CF809132048D7FB4CF809187
:1038900031048F7EA1CF809131048F7D9DCF8091A7
:1038A00031048F7B99CF01D9809131048F7794CFE8
:1038B00080913104837F90CF809132048C7F9BCFA5
:1038C00080913104992782FF939590FB82F990FBB8
:1038D00083F982CF80913204982F909590FB80F9E4
:1038E00090FB81F988CF90913104892F8F7B96FFCF
:1038F000806472CFDAD890913104892F97FB87F9D1
:1039000080586ACF61E08EE090E00E94C93166CFB6
:1039100060E0F9CF90913104892F8F7E94FF806110
:103920005BCF90913104892F8E7F90FF816054CFBF
:1039300090913204892F877F93FF88605CCF89E262
:1039400059C30737FCE71F0709F061C081E00E94F7
:1039500001087FC09272F801E052F847EB30F105A0
:1039600008F051C0E057FD4C0C94CD308091DD0340
:1039700080FF11C08E7F8093DD038DED93E00E9468
:103980005C110E9449088091DB0381608093DB0316
:103990000E94C30EE5CE81608093DD0361E08695D1
:1039A00086951ADCDDCE911521F05CDCD9CE91151F
:1039B000E1F34EDCD5CE911529F00E942312D0CE32
:1039C0009115D9F30E941B12CBCE911529F00E94BC
:1039D0003612C6CE9115D9F30E942B12C1CE911585
:1039E00029F00E944C12BCCE9115D9F30E944112CD
:1039F000B7CE911529F00E949811B2CE9115D9F346
:103A00000E948E11ADCE07372CE71207F9F0083768
:103A10003CE7130721F19801205E32452032310541
:103A200020F581113AC00F7181E090E0AC0102C035
:103A3000440F551F0A95E2F78A01642F83E090E056
:103A40000E94C931802F0E9479048ACE81E00E94B1
:103A5000F70743E062E081E00E942A0881CE8115E9
:103A600011F082E0F4CF82E072CF8115B1F00A3517
:103A70005CE7150709F4A2C008F079C001309CE7A3
:103A8000190709F499C00330ACE71A0709F48EC08E
:103A90000115BCE71B0709F47CC0F5018581E080B6
:103AA000F180811509F48EC0C7010E94190E182FEC
:103AB000682FC7010E947C04B701812F0E94FE0D70
:103AC0000E94F605F82E192FD5011596DC90159752
:103AD0001696CC90C2948FE0C8228091EB03877039
:103AE000811509F1ED2CD114F9F0892F807F8034F4
:103AF00069F080E28F0D8830B0F0892F807E8032AF
:103B000029F4B2E0FB1678F0C11469F08091320418
:103B100082FF09C082E00E940F088091EB0387704A
:103B2000EE24E3948111E12C812F82958F708830EF
:103B300009F454C108F067C0843008F048C0012F70
:103B40000F70823008F470C0107F103211F00295AF
:103B5000007FF11409F49EC0F1E0FF1609F400C1E2
:103B6000D11409F40CC1C11409F4B2C072C00B35F0
:103B7000ECE71E0729F180913204002482FF0394B0
:103B8000802D0C35FCE71F0709F087CF0E94E30B5F
:103B900084CF0E9455152FEF34E34CE02150304084
:103BA0004040E1F700C000000E94230B6FEF7FEF61
:103BB00080E090E00E94E3310E94751581E0E6CF3D
:103BC00080E0E4CFC7010E94B204182F75CF843083
:103BD00009F4E7C0E11409F430C18091EB0380FDE2
:103BE0002CC1D50115961C928695869586950E94C6
:103BF000F707C501A7DB8091EB038695869586952F
:103C00000E9401081AC1893009F45BC18A5F8F7074
:103C1000823000F7E2EFFE1265C1812F8F71D11063
:103C20005EC10E94F70707C1103110F00295007FB6
:103C3000D114B9F0011569F080E28F0D883010F0D1
:103C4000F11009C08091E603802B8093E6030E9467
:103C500096138F2D2FC08091EA03802B8093EA0367
:103C6000F6CF8F2D0E944E14011509F4B3CF80E2D8
:103C70008F0D883010F0F11004C0802F0E94F004E6
:103C800006C000958091EA0380238093EA030E9496
:103C90009613A0CF8091320482FD16C0D11469F032
:103CA000011539F08091E603802B8093E6030E9492
:103CB000961380E00E94EA138DCF80E00E944E149C
:103CC000011509F487CFD9CFD11469F1C11004C00F
:103CD000802F0E9433157ECF21E0C21211C01091B7
:103CE000E503802F8123081709F474CF0E94501335
:103CF0009093EF038093EE03102B1093E5036ACFAC
:103D000035E0C31267CF802F0E943315802F2BDA46
:103D10008091E703902F9823091709F45BCF802B3C
:103D20008093E70357CFC11011C0802F0E943C152C
:103D3000802F19DA8091E703902F9823911509F4C9
:103D400049CF009508230093E70344CF41E0C41214
:103D500041CF8091E6038023811509F43BCFE5CF65
:103D6000D11429F056E0C51608F034CFB1CF85E064
:103D7000C81608F02FCF802F0E943C152BCFC114FE
:103D8000D1F399E3F91209C0AFEFB7EEE3E0A15028
:103D9000B040E040E1F700C000008F2D0E944E14BB
:103DA00019CF812F869586958370811569F08130B2
:103DB00009F010CF8F2D912F9370D11002C080E0A9
:103DC00090E00E94B50806CF8F2D912F9370D110EF
:103DD00002C080E090E00E948D08FCCE812F8370AD
:103DE000811138C0D11027C04F2D4295469547709C
:103DF000440F440F8F2D8F70042E01C0880F0A943A
:103E0000EAF72F2D2071F4FE07C02FE030E001C04B
:103E1000220F4A95EAF720951695169513701230E1
:103E2000A1F0133081F03091E803113059F0822B6A
:103E300083230E9479040E947A0860E0C5010E94F1
:103E4000430E9FCC832B822BF4CF822B9091E803DF
:103E50008927EFCFD11451F110FFEDCF4F2D4295AF
:103E600046954770440F440F8F2D8F70042E01C06C
:103E7000880F0A94EAF72F2D2071F4FE07C02FE077
:103E800030E001C0220F4A95EAF720951695169565
:103E90001370123089F0133069F03091E90311305A
:103EA00041F0822B83230E94F307C5CF823018F2A2
:103EB000D5CF832B822BF7CF822B9091E9038927D3
:103EC000F2CF1F70D11439F0812F0E94F7078F2D88
:103ED0000E943315B0CF8F2D0E943C15812F0E9478
:103EE0000108A9CFF3EFFF1680F420EFF216E1F0FE
:103EF00031EFF316A1F0D11409F45FC0C11409F435
:103F000059C08F2D0E94EA1396CF43EFF416F1F0BB
:103F100054EFF512F0CF8091320482FD23C0812F3F
:103F20008F71D114E1F27DCED11469F085E0C8160D
:103F300008F081CF1F7181E090E0012E01C0880F51
:103F40000A94EAF7BACF96E0C916F2CF80E0D1140E
:103F500009F4A9CF1F7181E0012E01C0880F0A94D6
:103F6000EAF7A1CFD114B9F08091EB0387708430C8
:103F700049F41092EB031092ED031092EC03812FA1
:103F80008F71ADCFA5E063E0CA1608F054CF812F42
:103F90008F71D3D850CFB5E0CB1640F01092EB0321
:103FA0001092ED031092EC0364E0F1CF81E00E94E7
:103FB0000F0841CF812F8F7134CEC11401F3E9E393
:103FC000FE1209C0FFEF27EE33E0F15020403040F1
:103FD000E1F700C000008F2D0E944E142CCF063157
:103FE000BCE71B0709F0ADCC8091D803811509F41B
:103FF000A6CC85E30E94110914C09091E603063116
:10400000ECE71E0709F0A6CC9A7A81E0911101C075
:1040100080E08093D80385E3911101C089E20E947A
:10402000DD080E9496139CCBA0E0B0E0EAE1F0E24C
:104030000C94823080913004803108F048C0809127
:104040002F04811509F443C0C091F10387E0D82EF5
:104050008091F0038C17D9F1EC2EF12CDC9EE0015D
:104060001124FE01EE50FC4F84818115A9F191814C
:1040700080912B04981330C0908180912A0498136A
:104080002BC08581811128C00281138180912C046D
:1040900090912D04081B190B60E08AE294E00E94C5
:1040A000430E0E946C1208171907B0F48091300477
:1040B0008F70806180933004C850DC4F88818F708E
:1040C000806188838AE294E03DD90E94E604CDB7FE
:1040D000DEB7E7E00C949E30E7012196C770B8CFB9
:1040E000ADE0B0E0E6E7F0E20C947A308C0186E0D7
:1040F000F801DE01189601900D928A95E1F7F8011A
:10410000F580E4808AE2882E84E0982E80912E0447
:10411000811117C0E11491F0F11409F44FC1C801E5
:104120000E946E0E811509F449C187E0F801AAE2E8
:10413000B4E001900D928A95E1F776DFFF24F394C5
:1041400060C0A280B380D0902F0480912C04909105
:104150002D043501681A790AD11409F4EAC0C08027
:10416000518060E08AE294E00E94430E0E946C124B
:104170006816790608F09AC0E11401F380912B04C7
:10418000F8019181E0903004F0E1EF1608F059C099
:10419000981316C090912A04F8018081981310C0DA
:1041A000F11049C08E2D8F708061809330048AE2B7
:1041B00094E0C8D880913004F8018683F12C21C0A6
:1041C000F11039C040E0652D8C2D0E94DE0A40E0E0
:1041D000652D8C2D0E94DE0AF82E8111EFCF888587
:1041E00099850E94610E292F22952F70903470F4CA
:1041F0009F70223098F09115A9F0F80196819031C6
:1042000088F48F2D2D96EFE00C9496302A5F2F7056
:10421000223060F0C80196D8FD2CF3CF911511F033
:10422000811579F3805E883060F3F4CF803F48F3E6
:10423000815F8330F9CF80913004816080933004B6
:10424000BDCF981314C090912A04F801808198136F
:104250000EC0F1100CC0E682C80174D887E0F801E6
:10426000AAE2B4E001900D928A95E1F767CFC80108
:104270000E946E0E811509F4A1C0F11409F49EC0CC
:1042800080913004803208F450CF80912A049091BC
:104290002B049A838983BC82AB8280912E048D8308
:1042A0001E82EF82CE0101964DD83FCFD0903004D0
:1042B000F0E1DF1648F48AE294E044D887E0F401A4
:1042C00011928A95E9F77ACFE11409F437CF9091EA
:1042D0002B04F8018181981310C090912A048081E9
:1042E00098130BC0F11009C0D682C8012BD887E003
:1042F000F40111928A95E9F721CFC8010E946E0E50
:10430000811509F45BC0F11409F458C080913004A0
:10431000803208F40ACF80912A0490912B049A836A
:104320008983BC82AB8280912E048D831E82DF82C2
:10433000B9CF60E08AE294E00E94430E0E946C12C2
:104340006816790608F0BACFE11409F4F7CEF11433
:10435000A9F190912B04F8018181981325C09091C7
:104360002A048081981320C080912C0490912D0400
:10437000A81AB90AF8ECAF16B10408F06FCF809113
:10438000300480FD6BCF803108F468CFF80186835C
:10439000982F907F903F09F45FCF982F907F905F88
:1043A0008F70892B868358CFC8010E946E0E8111B1
:1043B000BCCE80913004816080933004C8010E949B
:1043C000A219BCCEABE1B0E0E8EEF1E20C9485308E
:1043D0004E8B5F8B688F798F8A8F192F9B8F9111EE
:1043E0001092EA031D8A86E0FE017696DE011F9692
:1043F00001900D928A95E1F70A8D8091320482FF37
:104400001FC00E9450132091EC033091ED03821BDA
:10441000930B8838934138F08091EB0382FD03C001
:1044200082E00E940F080E9450132091EE03309109
:10443000EF03821B930B8838934110F00E94F8041D
:10444000011561F00B8B1C8B61E0CE010F960E9471
:10445000430E61E0CE010F960E94430E0B8B1C8B26
:1044600087E0FE013F96DE01189601900D928A9535
:10447000E1F7CE01089634DE811110C02091F003DF
:104480003091F10387E0FE013896DE01119601902C
:104490000D928A95E1F78C8581110BC017E0809110
:1044A000F1039091F00389132BC06B96E4E00C9418
:1044B000A130822F90E0019687709927381719064E
:1044C00071F40E9455151092F0031092F10387E0E9
:1044D000EAE2F4E0DF011D928A95E9F7DFCF97E089
:1044E000929FD0011124AE50BC4FFE013196019035
:1044F0000D929A95E1F78093F0030E94E604CECFE7
:10450000189FC00111248E509C4FEADD811569F27D
:104510008091F10390E00196877099278093F103D1
:10452000BECFA6E0B0E0E7E9F2E20C9485300E944D
:1045300050138C0180910B0390910C03801791070D
:1045400071F019821A820E945013BC0149815A816C
:1045500080E090E037DF10930C0300930B03269666
:10456000E4E00C94A130A6E0B0E0E9EBF2E20C94B8
:1045700085308C019093080380930703011580E236
:104580001807B0F4C801805E9109089728F062E42A
:1045900075E10115110511F463E375E1C8010E948D
:1045A0004D04802F0E94EA132696E4E00C94A1307B
:1045B00080EF89838A830E9450138160BC01498106
:1045C0005A8181E091E0FEDEEFCFA6E0B0E0EBEEB5
:1045D000F2E20C9485308C019093080380930703DA
:1045E000011580E21807B0F4802F0E944E14C80114
:1045F000805E9109089728F06BE475E101151105BB
:1046000011F46CE375E1C8010E944D042696E4E0C4
:104610000C94A13080EF89838A830E9450138160BB
:10462000BC0149815A8181E090E0CCDEEFCFCF938D
:10463000DF93D82FC92F97DF8D2F9C2FC6DFDF91F7
:10464000CF9108950F931F93CF93DF938C01862F03
:1046500069E473E00E945712892B91F4C0914903D9
:10466000D0914A03209761F0F8018281833039F4B8
:10467000CE01DDDFCE01DBDFCE01D9DF01C0E0F707
:10468000DF91CF911F910F9108950F931F93CF93B7
:10469000DF938C01EB0169E473E08C2F0E945712C9
:1046A000892B09F057C0FE01FF27D80112968C9183
:1046B0001297E858FD4F8130A9F415968C9182FD30
:1046C0004EC080FF4CC082E0808380914B0390916C
:1046D0004C030097B9F48091490390914A030097E5
:1046E000C9F110C08230A1F515968C9182FD26C0CB
:1046F00080FD0AC083E0808380914D0390914E033A
:104700000097F1F030DF26C084E0808380914F0372
:10471000909150030097B1F78091490390914A031B
:10472000009701F184DF80914B0390914C03009737
:1047300049F78091490390914A03E4CF85E0808353
:104740008091490390914A03009721F070DFF1CFE7
:1047500086E08083DF91CF911F910F91089581E0D2
:104760008083B9CF80914B0390914C03B8CF0F93C6
:104770001F93CF93DF938C01EB0169E473E08C2FDF
:104780000E945712892B71F4DD27C858DD4F8881AC
:10479000F801128218828330E9F048F4813059F030
:1047A000823081F0DF91CF911F910F910895843075
:1047B000B1F08530B9F78091490390914A03009791
:1047C00089F306C080914B0390914C03009799F3B5
:1047D000FCDEE8CF80914D0390914E03F7CF80919E
:1047E0004F0390915003009799F72091490330911E
:1047F0004A0380914B0390914C0321153105F9F246
:10480000009731F7C901E4CFA4E1B0E0EAE0F4E2B7
:104810000C947C30FE013D9688E0DF011D928A9564
:10482000E9F789E8A82E81E0B82E8F014F01EE2428
:10483000E394F12C23E9C22E21E0D22EF5018191DF
:104840005F018F3F09F43EC0F894E82FE295EF70C6
:10485000F0E021A18F70A70102C0440F551F8A9577
:10486000E2F7CA01922F982B91A392A180958923F8
:1048700082A3789400C0EDE8F1E031E0712C219141
:104880002F3F79F0A22FA295AF70A05EB0E08C917F
:1048900090E02F7002C0959587952A95E2F780FFEA
:1048A0007FC080E0782A330FCE16DF0641F7F5018E
:1048B00082918F3F11F00E94F40650EA5A95F1F769
:1048C000D8017C920F5F1F4FBDE8AB16B1E0BB066D
:1048D00009F0B4CF48E050E0B4018DEB92E00E94C3
:1048E0007B319C01892B41F088E0F401ADEBB2E013
:1048F00001900D928A95E1F70091C60210E00A51ED
:104900001D4F232B09F44EC081E0809335020E9495
:104910005013909334028093330280910503FE017B
:1049200031967F01811509F498C084E0DF011D9262
:104930008A95E9F7809136028A3008F057C04AE933
:104940005CE0B701C8010E94A90B811509F473C08E
:1049500049E25DE0B701C8010E94A90B811509F485
:104960006AC048E65DE0B701C8010E94A90B811545
:1049700009F461C0109236028091C50290E044E0D3
:1049800050E0B7018A519D4F0E947B3121E0209376
:104990003202892B09F041C06496EDE00C94983006
:1049A000832F80CF80913502811509F4B6CFE09036
:1049B0003302F09034020E9450138E199F0905971C
:1049C00008F4ABCF44E050E06DEB72E0C8010E9408
:1049D0007B31892B41F084E0EDEBF2E0D8010190CE
:1049E0000D928A95E1F71092350297CFC090300270
:1049F000D09031020E9450138C199D09843F914040
:104A000008F09DCF80913202811531F284E0F701E8
:104A100011928A95E9F710923202E091C502F0E016
:104A2000EA51FD4F89819A81AB81BC81808391835A
:104A3000A283B383B1CF809136028F3F39F40E94B5
:104A400050139093310280933002DCCF8F5F8093BC
:104A500036028A3008F490CFF2CFF801808191813C
:104A6000A281B3818093380490933904A0933A04CF
:104A7000B0933B0488E394E00E943B0A80933704A0
:104A800080903C0490903D04A0903E04B0903F0480
:104A900080912C0290912D02A0912E02B0912F02B4
:104AA00088169906AA06BB06B1F080922C02909255
:104AB0002D02A0922E02B0922F020E944009861A67
:104AC000970AA80AB90A8092010390920203A09261
:104AD0000303B09204038CE0E0E4F4E0D70101901A
:104AE0000D928A95E1F7F0904104E0904204D09055
:104AF00043040091490410914A0480914B041092A0
:104B00004A04111509F448CF14FD8093DC0310FF0B
:104B10000DC0898180FF1EC09091DD03916090934C
:104B2000DD0360E0869586950E94EC1811FF06C0B3
:104B300020E04D2D6E2D8F2D0E94A21112FF04C07A
:104B4000011559F00E94D11813FF26CF81E0809300
:104B5000DE0222CF0E94E00FE9CF0E944908F4CF85
:104B6000CDB7DEB7AC970FB6F894DEBF0FBECDBFA2
:104B700085B7806885BF85B7806885BF84B7877F24
:104B800084BF0FB6F894A8958091600088618093E7
:104B90006000109260000FBE80E890E00FB6F894BD
:104BA00080936100909361000FBE81E080934E017D
:104BB00082EF96E090930302809302020E945008D5
:104BC0000E940E0A0E94840A8091E2008460809311
:104BD000E20078948091F002811599F08091E900CB
:104BE0001091EC008F70179511271795182B1092C4
:104BF000E9008091E80083FD0E948A151F701093E0
:104C0000E90082E084BD93E095BD9AEF97BD809363
:104C10006E0010920103109202031092030310928F
:104C200004030E94AA0E811102C00E94C212809148
:104C3000D80080618093D8002AE12A95F1F700C05E
:104C40008091D900182F117080FD04C00E940E0AB7
:104C50001092F0021093050353985B988FE891E04F
:104C60000197F1F700C0000089B183FB992790F903
:104C7000909306039093160183FD9EC086E0809377
:104C8000110186E0809312018091050381110E9439
:104C9000512E809116018091160191E08927880F8D
:104CA000880F8093C60294E0981B9093C50281E31D
:104CB0000E94F40683E30E94F40687E90E94F4064A
:104CC00084E30E94F4060DE811E0B3E9EB2EB1E0B5
:104CD000FB2ED8018D918D018F3F11F00E94F406BB
:104CE000E016F106B1F788E0E6EEF2E0DF01282FEA
:104CF0001D922A95E9F7EDEBF2E0DF011D928A950E
:104D0000E9F780E090E00E94B531833E9E4F21F4A8
:104D10000E94AA0E81112BC063EE7EEF80E090E02E
:104D20000E94E33160E082E090E00E94C93181E0BE
:104D30008093E80361E083E090E00E94C93160E085
:104D400074E184E090E00E94E3310E947D110E94B2
:104D5000C21240E050E0BA018FE090E00E94DB31E7
:104D600040E050E0BA0183E190E00E94DB3182E054
:104D700090E00E94A8318093CE0284E090E00E94EF
:104D8000B53190933204809331043EDDEFEFF6E7C6
:104D900021E0E150F0402040E1F700C0000034DDA8
:104DA0008091E60280FF0AC06FEF7FEF80E090E025
:104DB0000E94E3310E94230B80E061CF83E090E00A
:104DC0000E94A8310E9479048091E9030E94D007D3
:104DD0008091C702811125C08DED93E00E94E712FA
:104DE0008091DB0383608093DB038091DD0384305B
:104DF00030F40E947D118DED93E00E94E7120E9435
:104E0000A6070E9449080E9468088091DD0380FF80
:104E100005C060E0869586950E94EC1881E080933D
:104E2000C70280910503811103C082E30E94B02F65
:104E300089EA96E09093C9028093C80287E191E0E5
:104E400090932E0380932D038091F0028530D9F446
:104E50008091F002853009F460C00E9455150E94CF
:104E60007A081092CC028091CB02811551F080918A
:104E7000DD0381608093DD0360E0869586950E9466
:104E8000EC180E94D118C0DC0FEC12E0A6EEEA2E5E
:104E9000A2E0FA2ED701F80191918D9122E0E73D31
:104EA000F20709F47FC09817B9F380900503D12C5D
:104EB000D701CD907D01F80191908F019C1431F1C3
:104EC0009C24B12CAA24A394892D8A218115B9F0A0
:104ED0008114A9F0B982DA820E9450139C838B83DB
:104EE000F1E0FD8391E08C2D8A21811101C090E0D9
:104EF0009E8349815A816B817C818D8163DAB39471
:104F0000AA0C26E0B212E0CFF801C292D39438E0A6
:104F1000D312CECF0E944C0948C08091F002843059
:104F200009F434C00E9449088091CC0281110AC062
:104F300031E03093CC028091DD0381708093CB020D
:104F40000E94E00F1092CA0288E190E0A0E40FB640
:104F5000F894A895809360000FBEA093600083B77B
:104F6000817F846083BF83B7816083BF7894889595
:104F700083B78E7F83BF0FB6F894A89580916000A9
:104F8000886180936000109260000FBE3DDCE6EE09
:104F9000F2E081918111BDC42EEE32E02E173F0761
:104FA000C1F756CF981381CFBCDA809105038115E4
:104FB00071F1E090D303F090D403E114F10439F1DE
:104FC000C090D503D090D6030E9450138C010C19C9
:104FD0001D09C7010E946C1280179107C0F420912F
:104FE000D3033091D403C9019927287F3327232B7A
:104FF00009F0CEC0F4E0880F991FFA95E1F78D5AB9
:105000009C4FDC0115962C9122FF0E94751880910F
:10501000DA03811509F466C08091D903E091DD03BC
:10502000E695E695E81BE093DD02823009F0B3C017
:10503000F0E0E154F94FE4910E2F10E0EFE1CE2EB5
:10504000E0E1DE2E8091DE02811561F01092DE0239
:105050000E94C8189093DC028093DB021092E00259
:105060001092DF020E94C8189C018091DB0290918F
:10507000DC02A901481B590B4F3F5F4798F540914F
:10508000DA024115B1F01092DA024091D802509143
:10509000D902241B350B2F3F3F4758F4405D5A4837
:1050A0005093D9024093D8022091DB0328602093CB
:1050B000DB03E090DF02F090E002800F911F9093FD
:1050C000DC028093DB028BED92E0F6010995809182
:1050D000DF029091E002892B29F4EF2819F0F1E02A
:1050E000F093DA028091D702811569F01092D7020D
:1050F0008091DA03811107C08091DD0360E086951D
:1051000086950E94EC180E947A089091E102891716
:1051100021F08093E1020E9440098091F0028430E6
:1051200009F092CE83E08093E9008091E80082FF4D
:105130008BCE8091E80090E085FF06C00E94DD09DB
:10514000811509F468C091E08091E8008B77809325
:10515000E800911509F478CE0091090310910A0333
:10516000E9810115110509F473C0EE3F09F093C000
:105170008A81833020F08550833008F08CC0EA812A
:10518000EE3008F088C0F0E0E556FD4C0C94CD30D0
:1051900080E090E036CF863059F4F0E0E454F94FE7
:1051A000E4910E2F10E072E3C72E70E1D72E4ACFA4
:1051B000893061F4E695F0E0E754F94FE4910E2F61
:1051C00010E066E3C62E6FE0D62E3CCF8F3059F448
:1051D000F0E0EA54F94FE4910E2F10E058E6C52EA6
:1051E0005FE0D52E2FCF00ED17E03DE0C32E37E076
:1051F000D32E8C3109F026CF8E2F63E0AFD7E92F65
:10520000F0E0ED54F94FE4910E2F10E04CE9C42E7C
:1052100040E1D42E17CF00E210E09E012F5F3F4FF8
:1052200079018091E80085FD0AC08091E8008B77C4
:105230008093E8000E94DD09811599F384CF809165
:10524000F100D7018D937D010150104051F77BCFC4
:10525000E43148F4E11551F0E150E33138F4F0E085
:10526000E755FD4C9AC7EE3F09F489CF8FEF89834C
:1052700012C01A8289E08B830EC08A81823081F04D
:105280008330B9F0813091F70E9440098CD76B834D
:105290007C838D839E83CE0101960E942D0AD4CDFE
:1052A00088E290E00E94A8311B821C821D828E83BE
:1052B000F2CF8091EE029091EF02892B61F388E0AA
:1052C000E6EEF2E0DE01139601900D928A95E1F789
:1052D000E2CF8A81823051F66B817C818D819E8103
:1052E00062D788E290E00E94C931D5CF4C816B81B2
:1052F0008A810E94CF0D9827892798279E838D83C6
:10530000CACF2D813E813227232732274C816B81E2
:105310008A810E94F90BBFCF0E944110BCCF8A81C5
:10532000823869F178F48038B1F0813809F0B3CF70
:1053300060E08B810E94EC188B81811115C00E9466
:10534000E00FA9CF833809F0A6CF20E04091E00319
:105350006C818B8106C020E04B816091DF038091DE
:10536000DE030E94A21197CF8091DD0381608093BC
:10537000DD0360E0869586950E94EC188CCF8B81CA
:105380008093E10388CF8A818238E1F060F480382D
:10539000A1F0813809F07FCF8091DD0380FF10C03C
:1053A0008695869568CF833809F075CF8091DE03A6
:1053B0008B838091DF038C836ECF8091E0035BCF82
:1053C00080E059CF8091E10356CF0E94A6078DED72
:1053D00093E00E945C115FCF80E18A835CCF82E022
:1053E0008A8387E048CF8C818D3108F054CF8A8042
:1053F0009B80982489249824A12CB12C8E010F5FC6
:105400001F4F7801E80EF11CE016F10609F443CFB6
:1054100080E0B7E08B16B2E09B06A104B10420F453
:10542000C40187509E4F94D7F80184830F5F1F4FAC
:10543000FFEF8F1A9F0AAF0ABF0AE6CF8091EE02F4
:105440009091EF02892B09F426CF8C818D3108F0E1
:1054500022CF882E912CA12CB12CCA80DB80DC2499
:10546000CD24DC24E12CF12C8E010F5F1F4F412C49
:10547000512C3201481459046A047B0408F00BCF04
:1054800027E0C21622E0D206E104F10438F4D80184
:1054900014966C91C60187509E4F7BD7BFEF4B1A75
:1054A0005B0A6B0A7B0AEFEFCE1ADE0AEE0AFE0AEF
:1054B0000F5F1F4FDFCF0E948712EDCE84E08DCFAC
:1054C0008C818D3108F0E7CE882E912CA12CB12C47
:1054D000CA80DB80DC24CD24DC24E12CF12C412C9F
:1054E000512C32018E010B5F1F4F481459046A047E
:1054F0007B0408F0D0CE80E0F0E8CF16F1E0DF06C4
:10550000E104F10418F4C601899622D7D8018D93DD
:105510008D01BFEF4B1A5B0A6B0A7B0AEFEFCE1AC5
:10552000DE0AEE0AFE0AE1CF2C81022F10E02D31B7
:1055300008F0B1CE8A819B819827892798272C0172
:10554000612C712C8038F1E09F0708F0A4CE822EE8
:10555000912CA12CB12C40E851E060E070E044199E
:10556000550966097709421751056105710508F467
:1055700092CE2091EE023091EF02232B09F03EC033
:105580001C0129E2220E311C80FBEE24FF24E0F8EE
:1055900080FF0BC08896DCD69D81892798278927B4
:1055A00081159C4711F48FEF8D83D501C401840DC3
:1055B000951DA61DB71D80FF19C0680161E0C61AC0
:1055C000D108CE0105968C0D9D1D9CA78BA7C1010E
:1055D000800F911FBDD6ABA5BCA59C9181159C47A2
:1055E00021F48FEFEBA5FCA580838601FE013196A7
:1055F000EE0DFF1D2FEFE016F10638F08E010F5F64
:105600001F4FC12CD12C760125C094818581811535
:105610009C4711F42483258362E0E60EF11C329648
:10562000EACF80E8481681E058066104710430F43E
:10563000D80114966C91C2018996ABD6BFEFCB1AF4
:10564000DB0AEB0AFB0AEFEF4E1A5E0A6E0A7E0ACD
:105650000F5F1F4FC814D904EA04FB0410F31BCEDC
:105660008091EE029091EF02892B09F414CECE01C5
:1056700001960E942D0AFFEF21EE34E0F150204008
:105680003040E1F700C0000095CB88E0EFE4F1E0A6
:10569000DE01919601900D928A95E1F7FE01329616
:1056A0008FE1DF011D928A95E9F786E0898388E022
:1056B0007F96DE01159608CE84E6898381E08A8391
:1056C0001B821C82E8CD8B819C81092E000CAA0BC9
:1056D000BB0B25E0880F991FAA1FBB1F2A95D1F786
:1056E000AC01BD01405E5F4F6F4F7F4F48175907B8
:1056F0006A077B0708F4CFCD8436E1E09E07A10559
:10570000B10508F0C8CD4536F1E05F0761057105C8
:1057100020F044E651E060E070E0481B590BBC010A
:105720006D53794FCE010196D0D5B5CD4AE150E009
:105730006FEF70E0CE010796F4D58091EE02898379
:105740000A831B821C821D8281E0B1CD81E090E042
:1057500090930A038093090382E390E09093E5021B
:105760008093E4020E9450139093E3028093E2023C
:1057700092CD0115110571F1D090E602E090E202A0
:10578000F090E3020E9450138E199F09853691050F
:1057900040F1D1FE26C0D0FE24C00E945013909349
:1057A000E3028093E2028091E4029091E502019786
:1057B0009093E5028093E402892B61F410920A032E
:1057C0001092090381E090E09093EF028093EE0243
:1057D00000E010E08091EE0289830A838091E40268
:1057E0004ACD82E390E09093E5028093E402F2CF09
:1057F0001092EF021092EE024ECD40E250E06FEFB9
:1058000070E0CE0101968DD546CD8B81813069F057
:10581000823011F181113FCDFE0132968FE1DF011F
:105820001D928A95E9F788E022CD8C819AE0F92EC5
:105830008E010F5D1F4FF8012F2D11922A95E9F768
:10584000B8010E9457128983F801DE011296019077
:105850000D92FA94E1F71FCD6C818AE0FE01359636
:10586000DE01919601900D928A95E1F789A19AA1A6
:1058700081153CE7930741F42091EE023091EF024D
:10588000232B11F480E090E09AA389A38BA19CA123
:105890008115ACE79A0741F42091EE023091EF02B6
:1058A000232B11F480E090E09CA38BA38DA19EA1FB
:1058B0008115BCE79B0741F42091EE023091EF0285
:1058C000232B11F480E090E09EA38DA38FA198A5D7
:1058D0008115ECE79E0741F42091EE023091EF0232
:1058E000232B11F480E090E098A78FA38FEF68300E
:1058F00060F4FAE06F9FB001112467557E4F4AE0D3
:1059000050E0CE01819663D580E089830E945008E3
:10591000C2CC8091CD02811509F49ACA30E139BD1B
:1059200062E169BD09B400FEFDCF8091D8008F7D92
:105930008093D8008091E00082608093E0008091A5
:10594000E00081FDFCCF0E94551582CA78941F9219
:105950001FB61F9211248F939F93AF93BF93809193
:105960004C0290914D02A0914E02B0914F020196CF
:10597000A11DB11D80934C0290934D02A0934E0245
:10598000B0934F02BF91AF919F918F911F901FBE17
:105990001F9018951F920F920FB60F9211242F93FC
:1059A0003F934F935F936F937F938F939F93AF93A7
:1059B000BF93EF93FF938091E10082FF09C0809134
:1059C000E20082FF05C08091E1008B7F8093E100BF
:1059D0008091DA0080FF24C08091D80080FF20C031
:1059E0008091DA008E7F8093DA008091D90080FF69
:1059F000A9C080E189BD82E189BD09B400FEFDCF67
:105A000081E08093F00280913B02811109C00E94E5
:105A10000E0A0E94840A8091E20084608093E20072
:105A20008091E10080FF1AC08091E20080FF16C0E3
:105A30008091E2008E7F8093E2008091E20080619D
:105A40008093E2008091D80080628093D80019BCD6
:105A500085E08093F00283E080934E018091E10025
:105A600084FF2FC08091E20084FF2BC080E189BDBC
:105A700082E189BD09B400FEFDCF8091D8008F7D01
:105A80008093D8008091E1008F7E8093E100809127
:105A9000E2008F7E8093E2008091E200816080933B
:105AA000E20080913A02811509F452C084E08093AB
:105AB000F0028091F002843009F052C082E08093BD
:105AC0004E018091E10083FF2CC08091E20083FFB2
:105AD00028C08091E100877F8093E10082E080937D
:105AE000F00210923A028091E1008E7F8093E100F3
:105AF0008091E2008E7F8093E2008091E2008061DD
:105B00008093E20042E060E080E00E94540A8091CD
:105B1000F00088608093F00081E080934E018093D4
:105B20004D01FF91EF91BF91AF919F918F917F9127
:105B30006F915F914F913F912F910F900FBE0F90FA
:105B40001F90189519BC1092F00210923B0268CF7A
:105B50008091E30087FF02C083E0A9CF81E0A7CF57
:105B600081E0ADCF1F920F920FB60F921124EF92EA
:105B7000FF920F931F932F933F934F935F936F93D6
:105B80007F938F939F93AF93BF93CF93EF93FF93A5
:105B900009EE10E0F8018081C091EC008F70C7958C
:105BA000CC27C795C82B108280EFE82EF12CF70187
:105BB0008081877F808378940E948A15F801108203
:105BC000F701808188608083CF70F801C083FF91E6
:105BD000EF91CF91BF91AF919F918F917F916F91F5
:105BE0005F914F913F912F911F910F91FF90EF90F7
:105BF0000F900FBE0F901F901895FF920F931F9359
:105C0000CF93DF93182FEB011092BC0084EA8093AE
:105C1000BC000E945013082FF92E8091BC0087FF12
:105C200028C08091B900887F883029F08091B90020
:105C3000887F803199F51093BB0084E88093BC0085
:105C40000E945013182F092F8091BC0087FF1EC09F
:105C50002091B900287F80E090E0283199F081E020
:105C600090E0203411F480E090E0919581959109C5
:105C700009C0802F9F2D0E943B19C817D90768F6CD
:105C80008EEF9FEFCDB7DEB7E5E05AC2812F902FA0
:105C90000E943B19C817D907B8F6F2CF8FEF9FEFD4
:105CA000F1CF1092B90088E48093B80008950F9363
:105CB0001F93CF93DF93EB018093BB0084E8809325
:105CC000BC000E945013182F092F8091BC0087FF41
:105CD00011C02091B900287F81E090E0283211F4B2
:105CE00080E090E0919581959109DF91CF911F918E
:105CF0000F910895CF3FDC0741F3812F902F0E9431
:105D00003B19C817D90708F78EEF9FEFEECF0F9317
:105D10001F93CF93DF93EC0184EC8093BC000E942F
:105D20005013182F092F8091BC0087FF08C0809165
:105D3000BB0090E0DF91CF911F910F910895CF3F6D
:105D4000DC0789F3812F902F0E943B19C817D907D0
:105D500050F78EEF9FEFEECF0F931F93CF93DF930C
:105D6000EC0184E88093BC000E945013182F092F87
:105D70008091BC0087FF08C08091BB0090E0DF915C
:105D8000CF911F910F910895CF3FDC0789F3812FA9
:105D9000902F0E943B19C817D90750F78EEF9FEF3D
:105DA000EECFA0E0B0E0E6EDFEE2A5C1682E962EB3
:105DB0005A01690178010E945013782E892E04310E
:105DC000110518F10F3F100719F1C80164E170E0E7
:105DD0007AD1162F072F612F702F862D0EDFEC0141
:105DE000892BC1F0FFEFEF16FF06A9F3872D982D41
:105DF0000E943B19E816F90670F784E98093BC000D
:105E0000CE01CDB7DEB7EEE092C111E000E0E3CF06
:105E100015E0FCCFB701892D4ADFEC018501CA0CE2
:105E2000DB1C0C151D0549F3209739F7B701F80164
:105E300081918F013CDFEC01F4CFA0E0B0E0E2E221
:105E4000FFE259C1982E862E6A01590178010E94FD
:105E500050133C010431110538F10F3F100739F19F
:105E6000C80164E170E02FD1162F072F612F702F2A
:105E7000892DC3DEEC01892BE1F0FFEFEF16FF0661
:105E8000A9F3C3010E943B19E816F90678F784E9E3
:105E90008093BC00CE011C161D0614F480E090E037
:105EA000CDB7DEB7EEE043C111E000E0DFCF15E093
:105EB000FCCFB701882DFBDEEC01892B41F76894FC
:105EC00090F80E945013782E892E84E1E816F10490
:105ED00038F1EFEFEE16FE0631F1C70164E170E034
:105EE000F2D0162F072F612F702F892D86DEEC013F
:105EF000892BD9F400E010E0F1E0AF1AB1080A15DF
:105F00001B05F8F4D7FDC3CFC70101DFEC0197FDF6
:105F100004C0F601E00FF11F80830F5F1F4FEFCF2A
:105F200011E000E0E0CF15E0FCCF8FEFE816F806B7
:105F3000D1F2872D982D0E943B19E816F90698F6A4
:105F4000D9CFD7FDA4CFC70107DFEC0197FD05C06E
:105F5000CA0CDB1CF60180839ACFCEEFDFEF97CF20
:105F60008093BA0085EC8093BC0008951F920F9235
:105F70000FB60F9211242F933F934F935F936F931C
:105F80007F938F939F93AF93BF93CF93DF93EF93C1
:105F9000FF938091B900982F987F9038F1F038F4F2
:105FA000911509F48DC0903699F081E034C0887E57
:105FB000883AD9F7E0913404F0E0EA5CFB4F808145
:105FC0008093BB00809134048F5F80933404EDCFC5
:105FD0001092330410923504E8CF8091330481117C
:105FE00039C08091BB0080933404809134048631A1
:105FF00078F11092340480E091E090933304409162
:10600000340420912401309125014217130609F030
:1060100090E0909335049091BC008295880F880F92
:10602000807C892B85688093BC00FF91EF91DF9184
:10603000CF91BF91AF919F918F917F916F915F9120
:106040004F913F912F910F900FBE0F901F90189579
:1060500081E0D2CFE0913404F0E08091BB00EA5CB3
:10606000FB4F8083809134048F5F80933404809150
:106070003504811509F499CFC0919301D091940111
:10608000A88188E0A802D0011124AD5DBE4F16960C
:10609000ED91FC911797309709F487CF14962D91C5
:1060A0003C9115972C0F3D1F11966D917C91129785
:1060B0006C0F7D1F13964C9113978C91099575CF9A
:1060C0001092BC0072CFAA1BBB1B51E107C0AA1FD4
:1060D000BB1FA617B70710F0A61BB70B881F991F89
:1060E0005A95A9F780959095BC01CD0108952F92FE
:1060F0003F924F925F926F927F928F929F92AF9258
:10610000BF92CF92DF92EF92FF920F931F93CF93A4
:10611000DF93CDB7DEB7CA1BDB0B0FB6F894DEBF3B
:106120000FBECDBF09942A88398848885F846E8461
:106130007D848C849B84AA84B984C884DF80EE80AB
:10614000FD800C811B81AA81B981CE0FD11D0FB6B4
:10615000F894DEBF0FBECDBFED010895992778E01A
:10616000880F991F961708F0961B881F7A95C9F714
:106170008095089597FB072E16F4009406D077FDBE
:1061800008D0A1DF07FC05D03EF4909581959F4F84
:106190000895709561957F4F0895EE0FFF1F05904C
:1061A000F491E02D09946927962769277827872796
:1061B00078270895002E083090F0982F872F762F9B
:1061C000652F542F432F322F22270850F4CF220F50
:1061D000331F441F551F661F771F881F991F0A957D
:1061E000B2F7002D089597FD1094002E083098F016
:1061F0000850232F342F452F562F672F782F892FA4
:10620000912DF4CF15949795879577956795579528
:106210004795379527950A95AAF71124002D0895DB
:106220008F929F92AF92BF92CF92DF92EF92FF92A6
:10623000CF93DF93EC01688179818A819B8161151D
:1062400071058105910521F464E279ED8BE597E014
:106250002DE133EF41E050E0D1D049015A019B01DB
:10626000AC01A7EAB1E4E6D06B017C01ACEEB4EF7F
:10627000A5019401EBD0DC01CB018C0D9D1DAE1D61
:10628000BF1DB7FF03C00197A109B0488883998358
:10629000AA83BB839F77DF91CF91FF90EF90DF9030
:1062A000CF90BF90AF909F908F900895B9CF80E02E
:1062B00091E0B6CFA0E0B0E080930001909301019F
:1062C000A0930201B09303010895FB01DC0102C019
:1062D00005900D9241505040D8F70895FC0141506F
:1062E000504030F001900616D1F73197CF01089554
:1062F000882799270895FB01DC0104C08D91019046
:10630000801921F441505040C8F7881B990B08951B
:10631000FB01DC0102C001900D9241505040D8F7C2
:106320000895DC0101C06D9341505040E0F708959D
:10633000DC01CB01FC01F999FECF06C0F2BDE1BD45
:10634000F89A319600B40D9241505040B8F7089534
:10635000F999FECF92BD81BDF89A992780B508952D
:10636000A6E1B0E044E050E0E5CFA8E1B0E042E0D3
:1063700050E0E0CFDC01A40FB51F4150504040F089
:10638000CB01840F951F2E9105D041505040D8F776
:106390000895262FF999FECF92BD81BDF89A0197F5
:1063A00000B4021639F01FBA20BD0FB6F894FA9A5D
:1063B000F99A0FBE08950396272FECDFEADF252F09
:1063C000E9DF242FE7CF0196272FE4DFE2CFDC01BE
:1063D000CB0102C02D9105D041505040D8F708950F
:1063E000262FF999FECF1FBA92BD81BD20BD0FB6F1
:1063F000F894FA9AF99A0FBE01960895052E97FB24
:1064000016F400940FD057FD05D024D007FC02D01D
:1064100046F408C050954095309521953F4F4F4F19
:106420005F4F089590958095709561957F4F8F4F40
:106430009F4F089531D0A59F900DB49F900DA49FBC
:10644000800D911D11240895B7FFF4CFF3DF821B57
:10645000930B0895A1E21A2EAA1BBB1BFD010DC0D0
:10646000AA1FBB1FEE1FFF1FA217B307E407F50704
:1064700020F0A21BB30BE40BF50B661F771F881FE0
:10648000991F1A9469F760957095809590959B0176
:10649000AC01BD01CF010895A29FB001B39FC0011F
:1064A000A39F700D811D1124911DB29F700D811D40
:1064B0001124911D0895F894FFCF6B16911697162D
:1064C00091169716EA160C179716131820182B1CFE
:1064D000911C331CFE1B021C371C061C3B1C471C5A
:1064E000121C8A1C161C4B1C1A1C4F1C731C1E1CD5
:1064F000531C7A1C231C581C601C0A1C3F1C0E1CBD
:10650000431C271C5C1C6A1C821C881CF81B2F1C4B
:10651000981CCB1BD11BAA1BC51BD71BDD1BE31B68
:10652000B61CD31CD71CDB1CE01CE51CEA1CEF1CB2
:10653000F41CF91CFE1C452B5C2B632B4B294B29AF
:10654000962BA62BB92BF82BFD2B4B294B294B292E
:10655000052C39293D296929762981298C298F29FA
:10656000C329E5293629302BEC29EF29F3291E2AE6
:086570005B2A5E2A602A942ACE
:106578000100000001020112131415161718191A48
:106588001B000C000C0C013D09890B9F0B6409A42E
:106598000B800B010000000000000000000001015A
:1065A80000000000000004020000000406000000D3
:1065B8000000000C0A00000000000000000100FAC2
:1065C8003AA06F21695C370044226D3B011901AC88
:1065D8000069028202A20200010202020206060605
:1065E8000909090909090F0F0F12121212121212C2
:1065F8001212121C1C1C1C1C1C31339734F4F56637
:106608003635953604E200E900EA00B500B600B771
:1066180000CD008301CC008A01920194012102235C
:106628000224022502260227022A02B300B4006FC0
:106638000070009F01CB019F02A002E200E900EA7E
:1066480000B500B600B700CD008301CC008A0192E6
:106658000194012102230224022502260227022A8C
:1066680002B300B4006F0070009F01CB019F02A02D
:0266780002001E
:00000001FF
